:020000040000FA
:10000000280F00201D01000025010000270100002D
:10001000290100002B0100002D010000000000005C
:100020000000000000000000000000002F010000A0
:1000300031010000000000003301000083090000CE
:1000400037010000370100009D2500003701000046
:1000500037010000370100003701000037010000C0
:1000600037010000370100000000000037010000E8
:100070003701000027020000550200003701000090
:1000800037010000E31E00003701000037010000C7
:10009000370100006F200000370100003701000029
:1000A0003701000037010000370100003701000070
:1000B0003701000037010000370100003701000060
:1000C0003701000037010000370100003701000050
:1000D0003701000037010000370100003701000040
:1000E0003701000037010000370100003701000030
:1000F0003701000000000000000000003701000090
:100100003701000000000000DFF80CD005F036F8E1
:1001100000480047E1070000280F002006488047FC
:1001200006480047FEE7FEE7FEE7FEE7FEE7FEE7DC
:10013000FEE7FEE7FEE7FEE7A94500000901000033
:1001400010B5FF4C0321204603F021FF0122114688
:10015000204603F05EFF4FF4004300223221204688
:1001600003F006FFF7480023A114406D020120466A
:1001700003F0EAFE00221146204603F023FF00228E
:100180000121204603F038FF0D2000F001FB20463E
:10019000BDE81040012103F0FABE2DE9F0411446FC
:1001A000E94A0D460699E64FD0701E4680374FF457
:1001B00000430022384603F0DBFE00233246B91428
:1001C000384603F0C1FE224629463846BDE8F041D4
:1001D00003F012BF38B5DA4C03218034204603F017
:1001E000D6FE01221146204603F013FF4FF40043D0
:1001F00000220221204603F0BBFE002211462046C9
:1002000003F0E0FE1920002300904022032118464D
:10021000FFF7C3FF0E2000F0BBFA2046BDE83840D0
:10022000012103F0B4BE1CB5C54C0020009020781D
:100230000190C00703D0204603F0C0FE0090C248E2
:1002400000994160012101702046BDE81C40032156
:1002500003F09DBE1CB500200090B94890F88000C6
:100260000190BA4CC0070DD0204603F0A7FE0090C5
:10027000B5498860012048702046BDE81C40032134
:1002800003F085BE0098F3E72DE9F84FAE4D68788E
:1002900000287DD005F11006E8780127AC4CD6F88F
:1002A00028804FF0050A4FF01909092854D2DFE8D9
:1002B00000F005FDFCFB3B5489AEFA00404604F01B
:1002C000CCFC06468846E06D04F0C7FC82468B46AF
:1002D000A06D04F0C2FC04468946A86804F072FCD4
:1002E00000229C4B04F06DFB22464B4604F069FB58
:1002F00052465B4604F0BEFA4346324604F05BFBCE
:100300004FF03332944B04F05CFB3246434604F02A
:10031000B1FA04F0CDFC8C490023103140228862F0
:100320000F210420009715E0A86804F04BFC002280
:10033000884B04F046FB012204F024FC04F0B8FCD6
:100340004146306504F014FAB0630023E0220F2127
:1003500005200097FFF721FF1EE1A86804F032FC9A
:1003600000227C4B04F02DFB04F0A2FC0146F0635C
:10037000B06B04F0FDF930647848016BD1B1804670
:100380008068B8B102F03DFA04F067FC744A00E0FE
:1003900008E1744B04F015FB07460C46F06A04F0C4
:1003A0005CFC3A46234604F06BFC03D2D8F82C00E0
:1003B00002F03FF8002309214FF480720620CDF8A7
:1003C00000A0C7E7E06B04F048FC80468946A06BBC
:1003D00004F043FC0746A8680C46400004F0F2FB1A
:1003E00000225C4B04F0EDFA3A46234604F0E9FAA9
:1003F00042464B4604F03EFA04F05AFC7064002377
:100400000F214FF4A0720720CDF800A0A2E7206AC8
:1004100004F023FC80468B46E06904F01EFC044691
:10042000A8680F46A0F1006004F0CCFB0022494B05
:1004300004F0C7FA22463B4604F0C3FA42465B4644
:1004400004F018FA04F034FCB0644FF4B0740023E4
:1004500022460F210820CDF800A0FFF79EFEA878C5
:100460000321401CB0FBF1F201FB12003E4FA870CB
:1004700020B101282CD0022829D14EE0002380226F
:100480000F210120CDF80090FFF787FE03F09AFCC2
:100490007065316904F032FC7ED2306904F0DDFB16
:1004A00000223B4603E0C6E0E2E09AE07CE004F094
:1004B000E1F904460F46706D04F0CFFB22463B463F
:1004C00004F0DEFB706D306166D203F0F0FB63E098
:1004D0000023A0220F210220CDF80090FFF75DFE3F
:1004E00003F047FCB065716904F008FC54D27069F0
:1004F00004F0B3FB1D4A1E4B04F0BCF904460F4642
:10050000B06D04F0AAFB22463B4604F0B9FBB06D87
:10051000706141D203F0EAFB3EE0002322460F2146
:100520000820CDF80090FFF738FE03F074FCF0656A
:10053000B16904F0E3FB2FD2B06904F08EFB19E03F
:10054000000003400402002000000020800003405F
:10055000680200200000443E3333D33FA001002056
:10056000CDCCCCCCCCCCEC3F0000F03F7B14AE47E4
:10057000E17A843F00223B4604F07CF904460F46B2
:10058000F06D04F06AFB22463B4604F079FBF06D07
:10059000B06101D203F0B1FB0121844803F0F7FC04
:1005A00000206870BDE8F88FA06904F056FB804613
:1005B0008A46606904F051FB81460C46A86804F045
:1005C00001FB00227A4B04F0FCF94A46234604F072
:1005D000F8F94246534604F04DF904F069FBF06225
:1005E00023E0A06A04F039FB82468946606A04F081
:1005F00034FB04468846A86804F0E4FA00226C4BF9
:1006000004F0DFF92246434604F0DBF952464B463C
:1006100004F030F904F04CFB66493063884202DD97
:1006200002F00EF801E002F011F80023C0220F21C1
:10063000032000978EE6206D04F00FFB824689466A
:10064000E06C04F00AFB04468846A86804F0BAFA95
:100650000022574B04F0B5F92246434604F0B1F9A5
:1006600052464B4604F006F904F022FBF064DCE746
:10067000B06C20F0004004F0F0FA0446706C0F46B5
:1006800020F0004004F0E9FA80464B488A46406971
:1006900004F0E3FA4246534604F08DF90022474B3A
:1006A00004F08FF922463B4604F08BF904460F46CE
:1006B000A86804F087FA00223D4B04F082F900227A
:1006C0003F4B04F078F900223E4B04F07AF92246C1
:1006D0003B4604F0CFF804F0EBFA3B4970638842E4
:1006E00002DD0C2002F077FEF169706B04F006FB6E
:1006F00014D2F06904F0B1FA344A354B04F0BAF878
:1007000004460F46706B04F0A8FA22463B4604F0FC
:10071000B7FA706BF06101D203F0F6FA00234022C1
:1007200003211846CDF8009014E670B5294CD4E9A1
:100730000A0104F023F804F090FA274A274B04F04A
:1007400040F921F000450646D4E9110104F016F8FD
:1007500020F0004004F081FA32462B4604F08AF87B
:10076000BDE8704004F0A4BA1A4810B5816D406D20
:1007700004F004F820F0004010BD10B5FFF7F4FFBE
:100780000446FFF7D2FF2146BDE8104004F028B828
:10079000002809DB00F01F02012191404009800080
:1007A00000F1E020C0F80011704700008000034015
:1007B0000000443E0AD7233C040200200000084009
:1007C0000000E03F000059400000E2427B14AE47C9
:1007D000E17A843F10000020FCA9F1D24D62503F25
:1007E00000220221104603F00FFE6E48002505800E
:1007F000858040F64251818543F6070181876A482A
:100800000570694834300580684C44F23C00208013
:100810004FF4284020860520A4F86000992020711C
:100820000C2084F83400207E40F01000207684F8FC
:10083000485000F0E5F801F001FC0A21052000F025
:10084000FAF8482003F040FB492003F03DFB4B2021
:1008500003F04DFBE2130021412001F03DFDFFF7C5
:100860006FFCFFF7B7FC03F0E8F903F019FA03F0A7
:1008700083F902F0C1FD03F0C9F903F05FFA02F059
:100880003EF801F0C7FE94F84400494E494CDFF8A9
:100890002881C0064FF47A773CD5356047487560AB
:1008A000C6E9025075614648C6E90775C16A454800
:1008B00003F096FF01F045FFDFF80C91484601F088
:1008C00087FF424820624248C4E909054148606008
:1008D0004148C4F81890C4E904504FF07F5002F02A
:1008E0007EFC4FF04040E0623C4820633C48A06002
:1008F0003C48E0603C4860633C48A0633C48C4E935
:100900000F0501206564C4E913504FF4E131C8F8C4
:10091000201001E002F0C8FF0321D8F8200000F009
:10092000C1F834480068B0FBF7F0401EB0F1807F9A
:1009300009D24FF0E02148612F4AE02082F8140DDF
:100940008D6107200861706901F035FEF06801F0E3
:1009500040FD0021306801F07FFE0121706801F048
:100960007BFE606902F03BF8606C02F01FF800BF8C
:1009700001F07FFA02F0D0FAFFF786FC03F058FA94
:10098000F6E71E48D0E90212491C42F10002C0E914
:100990000212D0E90812491C42F10002C0E9081213
:1009A00001F036BF002000401024004000600040ED
:1009B000A0010020040200207000002000009040F0
:1009C0006802002000007A4400002040000020411E
:1009D000CDCCCC3E00401C460000604000004040B2
:1009E00000409C4500606A46197F933AFC1C7639AA
:1009F00004F6B733C80200200FE000E0100000202A
:100A000010B51B4C0021204603F0C3FB4FF42841D6
:100A1000204603F0B3FB4FF0402400220321204680
:100A200003F03DFC20460222BDE8104040F6C533ED
:100A3000910303F02FBC70B50C4605460A21491EF0
:100A4000FDD14FF480524FF040265100304603F064
:100A500031FC2946304603F028FC210A304603F0D9
:100A600024FCE1B23046BDE8704003F01EBC00003B
:100A700030600040B0F5165F11D0B0F5964F0ED043
:100A8000B0F5164F0BD0B0F5614F08D0B0F5E13F8F
:100A900005D0B0F5613F02D0B0F5E12F01D13F495B
:100AA0000862704710B53D4B0A4600211960596035
:100AB0009960D960196159619961D9610B46384CC7
:100AC0000146204603F02EFC00220121204603F0BF
:100AD00082FC0321204603F08BFCBDE8104011206E
:100AE00000F04EB870B52E4A0D46032908D02B4CA5
:100AF000E168B1F5806F08D00126012D08D011E022
:100B00000146104603F05DFC22E06FF0010070BD6D
:100B10004FF0E0234FF40031C3F88011BFF34F8F43
:100B2000BFF36F8FE16949B12289E1681D4B0A4427
:100B3000C2F30902491C9854E16004E001461046E2
:100B400003F03FFCE661012D02D1112000F018F8FE
:100B5000002070BD10B50446002006E010460121BB
:100B6000641CFFF7BFFF002802D12278002AF5D1CC
:100B700010BD10B504460A4803F02BFC207010BDD0
:100B8000002809DB00F01F0201219140400980008C
:100B900000F1E020C0F80011704700007000002054
:100BA00000500040D803002008B5694605F092FFC8
:100BB00000990978002900D0FE4808BD38B50C46D8
:100BC000694605F087FF0099097819B10B2002F0FA
:100BD00002FC38BDA04738BD38B50C460022694636
:100BE000F54803F03AFD0099097819B10B2002F09D
:100BF000F2FB38BDA04738BD70B50022144612E0A4
:100C0000ED4901EB4215014608E0202B09D0092BE4
:100C100007D02C2B05D005F8013B491C0B78002B85
:100C2000F3D12C70521C002107E0202B03D0092B9C
:100C300001D029B900E00121401C0378002BF4D138
:100C400013F0FF0F01D0182ADADB104670BD2DE932
:100C5000F04FAFB0FFF7D0FFD74DD84C203502286A
:100C600002D0182817D0F7E0D348FFF79DFF0646BB
:100C70002846FFF799FF0546304601F097F900280E
:100C80007ED1284601F092F90028F9D12660C4E906
:100C90000165E5609DE1C848FFF786FF07462846E5
:100CA000FFF782FF1090C4484030FFF77DFF0F90A0
:100CB000C1486030FFF778FF0E90BF488030FFF7E3
:100CC00073FF8346BC48A030FFF76EFF8146BA48E9
:100CD000C030FFF769FF8046B748E030FFF764FF98
:100CE0008246B748FFF760FF0646B5482030FFF759
:100CF0005BFF0D90B2484030FFF756FF0C90B048B4
:100D00006030FFF751FF0B90AD488030FFF74CFF8C
:100D10000A90AB48A030FFF747FF0990A848C030C1
:100D2000FFF742FF0890A648E030FFF73DFF07902D
:100D3000A448FFF739FF0690A2482030FFF734FFA0
:100D40000590A0484030FFF72FFF04909D48603089
:100D5000FFF72AFF03909B488030FFF725FF0290A2
:100D60009848A030FFF720FF01909648C030FFF769
:100D70001BFF00909348E030FFF716FF054600E0A8
:100D80005AE0384601F012F9002862D1109801F0BB
:100D90000DF900285DD10F9801F008F9002858D10D
:100DA0000E9801F003F9002853D1584601F0FEF8DF
:100DB00000284ED1484601F0F9F8E8BB404601F062
:100DC000F5F8C8BB504601F0F1F8A8BB304601F079
:100DD000EDF888BB0D9801F0E9F868BB0C9801F0BC
:100DE000E5F848BB0B9801F0E1F828BB0A9801F040
:100DF000DDF808BB099801F0D9F8E8B9089801F0C6
:100E0000D5F8C8B9079801F0D1F8A8B9069801F04B
:100E1000CDF888B9059801F0C9F868B9049801F0CF
:100E2000C5F848B9039801F0C1F828B9029801F053
:100E3000BDF808B9019800E00BE001F0B7F840B93F
:100E4000009801F0B3F820B9284601F0AFF8002867
:100E50007DD00B2002F0BFFAE06D03F0FEFE83466A
:100E60002691A06D03F0F9FE81468A46606D03F07D
:100E7000F4FE07468846206D03F0EFFE05460E4659
:100E8000E06C03F0EAFECDE92401A06C03F0E5FE7E
:100E9000CDE92201606C03F0E0FECDE92001206C79
:100EA00003F0DBFECDE91E01E06B03F0D6FECDE9D9
:100EB0001C01A06B03F0D1FECDE91A01606B03F0B9
:100EC000CCFECDE91801206B03F0C7FECDE9160179
:100ED000E06A03F0C2FECDE91401A06A03F0BDFE92
:100EE000CDE91201606A03F0B8FECDE91001206A75
:100EF00003F0B3FECDE90E01E06903F0AEFECDE9EB
:100F00000C01A06903F0A9FECDE90A01606903F0B4
:100F1000A4FECDE90801206903F09FFECDE906019A
:100F2000E06803F09AFECDE90401606803F095FEE5
:100F3000CDE90201A06803F090FECDE90001206830
:100F400003F08BFE02460B461F48269900E00AE09C
:100F5000CDE92CB126A981E8E00701F02DF82FB0EA
:100F60000020BDE8F08F27601098A0600F986060A7
:100F70000E98C4E9030BC4E907A6C4E905980D98C7
:100F800060620C98A0620B98E0620A98206309984E
:100F900060630898A0630798E0630698206405984A
:100FA00060640498A0640398E06402982065019846
:100FB00060650BE00000C07FD807002068020020B9
:100FC000D8080020D80900209C6E00000098C4E9D1
:100FD000160502F0A7FB3FE710B5F7A1F8A000F057
:100FE000EBFF002010BDBFF34F8FF6480168F64AB3
:100FF00001F4E06111430160BFF34F8F00BFFDE7D3
:101000002DE9F04FF14C93B0206B03F026FE8046A3
:101010008A46E06A03F021FE83460A91E06803F005
:101020001CFE07468946A06803F017FE05460E46DB
:10103000A06A03F012FECDE90801606A03F00DFE1C
:10104000CDE90601206A03F008FECDE904016068DD
:1010500003F003FEDE4CCDE90201606803F0FDFD04
:10106000CDE90001206803F0F8FD0B460A9902461D
:10107000CDE9108ACDE90EB10AA880E8E002D5A03A
:10108000A16800F099FF002013B06AE72DE9F04F46
:10109000DE4C8FB0E06C03F0E0FD82468846206BAA
:1010A00003F0DBFDCDE90801C848006803F0D5FD79
:1010B00083460791606C03F0D0FD07468946A06C1B
:1010C00003F0CBFD06460391E06A03F0C6FD05463A
:1010D0000191A06A03F0C1FD0B4604A90296009598
:1010E00081E8800A0246BA48CDE90AA88168C8A00A
:1010F00000F062FF00200FB033E72DE9F04FB34C52
:10110000BBB0E06903F0A9FD36908A46206B03F07E
:10111000A4FD81463391E06A03F09FFD32900F46B3
:10112000E06803F09AFD80468B46A06803F095FDC9
:10113000CDE92D10A06A03F090FDCDE92B10606A77
:1011400003F08BFDCDE92910206A03F086FDCDE97F
:101150002710606803F081FD9D4ECDE92510F068F1
:1011600003F07BFDCDE92310706803F076FDCDE937
:101170002110306803F071FDCDE91F10706A03F093
:101180006CFD1E911C9002F023F93990606903F008
:1011900064FDCDE91A01206803F05FFD9B4DCDE9A8
:1011A0001801E86D03F059FDCDE91601A86D03F0B3
:1011B00054FDCDE91401686D03F04FFDCDE9120136
:1011C000286D03F04AFDCDE91001E86C03F045FD00
:1011D000CDE90E01A86C03F040FDCDE90C01686C6F
:1011E00003F03BFDCDE90A01286C03F036FDCDE9A3
:1011F0000801686B03F031FDCDE90601286B03F0AF
:101200002CFDCDE90401E86A03F027FDCDE90201D8
:10121000A86A03F022FD0D46009001F0ECFA0246A8
:10122000206CCDE937A033993397CDE93491CDE9DE
:10123000308B2D992F912B992D9129992B912799AD
:1012400029912599279123992591219923911F99D6
:1012500021911E991C98CDE91E0139981C90019589
:10126000636C7548B16800F0A7FE00203BB078E6DB
:101270002DE9F04F95B002F07CFD03F0EEFC634CDD
:1012800083461191606B03F0E8FC81468A46206B2F
:1012900003F0E3FC07468846E06A03F0DEFC0546FF
:1012A0004B480E46C06803F0D8FCCDE90801A06A9F
:1012B00003F0D3FCCDE906014448406903F0CDFCBE
:1012C000CDE90401606C03F0C8FCCDE90201A06C1B
:1012D00003F0C3FC00903D480C46006801F0A5FFF8
:1012E00003F0BBFC0B460AA9019481E8E00F02461B
:1012F00052A000F061FE002015B032E610B5FFF7F5
:101300007BFC18B15A495B48FFF766FC304881689E
:1013100059A000F051FE002010BD7CB5FFF76CFC19
:10132000012802D002280BD01EE05248FFF73CFCF7
:1013300020F00041C1F1FF41002912D400212BE02F
:101340004C48FFF731FC04464A482030FFF72CFC9C
:101350000546204600F02AFE18B9284600F026FE71
:10136000A0B10B2002F037F8194D686803F075FC46
:1013700004460E46286803F070FCCDE9004602469C
:101380000B463EA000F018FE00207CBD0021204648
:1013900001F062F90121284601F05EF9E4E71B48FB
:1013A00010B5806A03F059FC02460B4636A000F0E7
:1013B00003FE002010BD000056302E380000000053
:1013C000257300000CED00E00400FA050402002083
:1013D000A0010020257520252E336620252E33669A
:1013E00020252E336620252E366620252E366620B3
:1013F000252E366620252E336620252E33662025A1
:101400002E326620252E32660000000010000020DB
:10141000257520252E356620252E356620252E346F
:101420006620252E346620252E336620252E35662F
:1014300020252E356600000044700000252E3566FC
:1014400020252E356620252E356620252E35662052
:10145000252E356620252E356620252E356620253D
:101460002E356620252E356620252E356600000097
:1014700047250000D807002025750000252E33667B
:1014800020252E3366000000252E36660000000061
:1014900010B5FFF7B1FB18B1FD49FE48FFF79CFB03
:1014A000FD484169AFF2300000F086FD002081E781
:1014B00010B501F021F80146AFF2440000F07CFDC8
:1014C000002077E7F54810B5C06A03F0C6FB024676
:1014D0000B46AFF24C0000F06FFD00206AE710B53C
:1014E000FFF78AFB18B1EE49EA48FFF767FBEA48C5
:1014F000C06803F0B2FB02460B46EAA000F05CFDB8
:10150000002057E7E54810B5006D03F0A6FB024642
:101510000B46E4A000F050FD00204BE710B5FFF7AC
:101520006BFB18B1E149DB48FFF756FBDA48C169AC
:10153000AFF2BC0000F040FD00203BE710B5FFF724
:101540005BFB18B1DA49D348FFF738FBD248406A51
:1015500003F083FB02460B46D6A000F02DFD0020D1
:1015600028E710B5FFF748FB18B1D449C948FFF781
:1015700025FBC948806A03F070FB02460B46D0A0E9
:1015800000F01AFD002015E710B5FFF735FB18B184
:10159000CD49C048FFF712FBC048006C03F05DFB6B
:1015A00002460B46C6A000F007FD002002E710B57A
:1015B000FFF722FB18B1C549B648FFF70DFBB64847
:1015C000016BAFF24C1000F0F7FC0020F2E610B512
:1015D00001F011F90146AFF2601000F0EDFC0020BF
:1015E000E8E610B5FFF708FB18B1B949A948FFF7BD
:1015F000F3FAB848416CAFF2801000F0DDFC002037
:10160000D8E610B5FFF7F8FA18B1B349A148FFF7CB
:10161000E3FAB048016CAFF2A01000F0CDFC00205E
:10162000C8E610B5FFF7E8FA18B1AC499948FFF7DA
:10163000C5FAA848406803F010FB02460B46A0A07C
:1016400000F0BAFC0020B5E6A24810B5006803F02F
:1016500004FB02460B469AA000F0AEFC0020A9E66F
:101660002DE9FF41FFF7C8FA9A4C03281CD189489D
:10167000FFF79AFA074687482030FFF795FA0646A3
:1016800084484030FFF790FA0546384600F08EFC5B
:1016900038B9304600F08AFC18B9284600F086FCBC
:1016A000D0B10B2001F097FEE06B03F0D6FA0746AD
:1016B0008846A06B03F0D1FA05460E46606B03F036
:1016C000CCFA8DE8E00102460B4685A000F074FCE0
:1016D00004B00020BDE8F0816763C4E90E65E3E76C
:1016E00010B5FFF789FA80B16A48FFF75DFA20F07C
:1016F0000041C1F1FF41002904D401F0C5FD01F012
:1017000059FB02E00B2001F066FE7248406801F0D0
:101710008CFD03F0A2FA02460B4676A000F04CFCCA
:10172000002047E66B4810B5006801F07EFD03F02D
:1017300094FA02460B46AFF2B02000F03DFC0020C8
:1017400038E6564810B5806C03F087FA02460B461F
:1017500068A000F031FC00202CE610B5FFF74CFA31
:1017600030B15C48406C18B964494A48FFF726FA22
:101770004A48406C03F071FA02460B465DA000F047
:101780001BFC002016E610B5FFF736FA514C28B1C5
:10179000206D18B95A493F48FFF710FA606903F005
:1017A0005CFA02460B463FA000F006FC002001E672
:1017B00010B5FFF721FA18B152493648FFF70CFA75
:1017C0004448816CAFF2503000F0F6FB0020F1E5A8
:1017D00010B5FFF711FA18B14B492E48FFF7FCF985
:1017E0003C48016DAFF2703000F0E6FB0020E1E50F
:1017F00010B5FFF701FA18B144492648FFF7DEF9A2
:101800003448806903F029FA02460B4640A000F0F4
:10181000D3FB0020CEE510B5FFF7EEF918B13D4936
:101820001C48FFF7CBF92B48C06903F016FA0246B3
:101830000B46AFF2304000F0BFFB0020BAE510B518
:10184000FFF7DAF918B134491248FFF7B7F9214820
:10185000006A03F002FA02460B46AFF2D43000F001
:10186000ABFB0020A6E510B5FFF7C6F918B12B4970
:101870000848FFF7A3F91748406A03F0EEF902465B
:101880000B46AFF2FC3000F097FB002092E5000021
:10189000B7250000D8070020A0010020100000207C
:1018A000D3230000252E346600000000B12600007E
:1018B00043270000252E316600000000D1270000DC
:1018C000252E33660000000033240000EB240000C6
:1018D000AD29000004020020D3290000B52D00002E
:1018E000252E31306620252E31306620252E3130D0
:1018F00066000000252E3566000000001D2900004E
:10190000DF290000BF280000F3280000312A000072
:1019100025660000DF310000E12D0000032E0000ED
:1019200010B5FFF769F918B1FB49FC48FFF746F914
:10193000FB48806A03F091F902460B46AFF2B840CB
:1019400000F03AFB002035E510B5FFF755F918B166
:10195000F449F248FFF732F9F148806803F07DF965
:1019600002460B46AFF2A80000F026FB002021E55E
:1019700010B5FFF741F918B1EB49E848FFF71EF938
:10198000E748C06803F069F902460B46AFF2D000A1
:1019900000F012FB00200DE510B5FFF72DF980B126
:1019A000DE48FFF701F920F00041C1F1FF410029B5
:1019B00004D401F069FC01F08EFA02E00B2001F082
:1019C0000AFDD748C06801F030FC03F046F9024632
:1019D0000B46AFF2E00000F0EFFA0020EAE410B5A9
:1019E000FFF70AF980B1CD48FFF7DEF820F000419B
:1019F000C1F1FF41002904D401F046FC01F05BFA7B
:101A000002E00B2001F0E7FCC548806801F00DFC06
:101A100003F023F902460B46AFF2281000F0CCFA8F
:101A20000020C7E410B5FFF7E7F818B1BF49BB487D
:101A3000FFF7C4F8BA48C06A03F00FF902460B4634
:101A4000AFF2406000F0B8FA0020B3E410B5FFF741
:101A5000D3F818B1B649B148FFF7B0F8B048006BF9
:101A600003F0FBF802460B46AFF2686000F0A4FA00
:101A700000209FE410B5FFF7BFF818B1AD49A748A3
:101A8000FFF79CF8A648C06C03F0E7F802460B4647
:101A9000AFF2906000F090FA00208BE4A64810B5F9
:101AA000406B03F0DAF802460B46AFF2EC1000F0A0
:101AB00083FA00207EE4A04810B5006B03F0CDF857
:101AC00002460B46AFF2D41000F076FA002071E423
:101AD000994810B5C06C03F0C0F802460B46AFF24F
:101AE000EC1000F069FA002064E4934810B5C06D72
:101AF00003F0B3F802460B46AFF2582000F05CFA50
:101B0000002057E48C4810B5C06B03F0A6F80246DD
:101B10000B46AFF2702000F04FFA00204AE48648EE
:101B200010B5406D03F099F802460B46AFF23C2029
:101B300000F042FA00203DE47F4810B5806D03F0CC
:101B40008CF802460B46AFF2542000F035FA002024
:101B500030E410B5FEF7E9FD03F07FF802460B46CE
:101B6000AFF2702000F028FA002023E410B5FEF751
:101B7000FBFD03F072F802460B46AFF2882000F03E
:101B80001BFA002016E410B5FEF7F7FD03F065F828
:101B900002460B46AFF2A42000F00EFA002009E442
:101BA00010B501F047FF65A000F006FA00207EE4C2
:101BB00038B5FFF721F8654C022810D1574964A0C9
:101BC00002F025FD40B9554800226946203002F058
:101BD00044FD0099097841B10B2001F0FCFB5EA0A7
:101BE000216800F0E9F9002038BD206001F0F2FF23
:101BF000F5E738B5FFF700F8584C022810D14749EF
:101C000053A002F004FD40B9444800226946203048
:101C100002F023FD0099097841B10B2001F0DBFBB4
:101C20004DA0216800F0C8F9002038BD206001F007
:101C3000D1FFF5E710B5FEF7DFFF022807D13749DE
:101C400043A002F0E4FC48B10B2001F0C4FB44497E
:101C5000AFF6940000F0B0F9002028E42F482030BF
:101C6000044602F0CDFC1F28F1D821463C4802F082
:101C7000DCFC01F0AFFFEAE710B5AFF6C403334870
:101C80003749026837A000F097F900200FE410B53B
:101C9000FEF7B2FF022807D1204937A002F0B7FCB7
:101CA00048B10B2001F097FB3549AFF6EC0000F08E
:101CB00083F9002005E419482030044602F0A0FC16
:101CC0001F28F1D821462E4802F0AFFC01F0AEFFEC
:101CD000EAE710B5FEF790FF18B12A490F48FEF762
:101CE0007BFF2948016AAFF6700000F065F900201B
:101CF00007E42DE9F04788B0FEF77EFF0E4C40B1B7
:101D0000064922A002F083FC20B10B2001F063FB06
:101D10006EE04EE03EE000004F2E0000D8070020AD
:101D200004020020B72E0000D72E0000712E000004
:101D3000952E0000F72E000010000020636F6E66E5
:101D4000696720736176656400000000600200200E
:101D50007361766500000000256C75006402002048
:101D6000E80A00204B6F6865726F6E2C25732C2576
:101D7000752C2573000000007772697465000000FF
:101D8000080B0020750A0000700000207265736562
:101D9000740000000025256001F082FF0021A16091
:101DA000C4E903156561A5618AA0E56100F004F945
:101DB0001EE0E06902F051FF80468946A06902F00A
:101DC0004CFF82460F46606902F047FF05460E460B
:101DD000206902F042FF02460B468DE86C0405A81C
:101DE00080E88003D4E902237EA0216800F0E4F8B3
:101DF00008B00020BDE8F08710B501F0E9FA01460F
:101E00007EA000F0D9F800200AE438B5FEF7F4FE11
:101E100068B1102269467A4802F01FFC0446009817
:101E2000007830B10B2001F0D6FA002105E04FF028
:101E3000FF34204601F0D6FA214670A000F0BCF82D
:101E4000002038BD10B501210D20FEF74BFE040027
:101E500007D101210A20FEF745FE044669A0FEF7DE
:101E600079FE72B6002068494861486062B6204633
:101E700057E42DE9F0416448416901292FD1816976
:101E800021B100218161BDE8F041DBE75F4E002414
:101E90005F4D604F08E000BF57F824100422304621
:101EA00002F0CCFB28B1641C55F824000028F3D1C3
:101EB00009E055F8244034B157A0FEF74BFE5348D3
:101EC000001DA047DFE7514802F09AFB0028DAD056
:101ED00052A0FEF73FFE0A2001F07DFAD3E7BDE8ED
:101EE000F081F8B5534802F086FA80B2C10747D1B5
:101EF00000F0060001260025434C022841D00428AA
:101F00003ED16846FEF735FE6069404F00289DF8D7
:101F1000000008D00D2831D00A282ED0012001F071
:101F20005AFAA6612AE008280DD00A2826D00D28E2
:101F300016D07F2807D061687854491C6160B1F5DC
:101F4000807F0FD013E06168C1B1491E61607D548C
:101F50000221FEF7C7FD02212020FEF7C3FD06E0A7
:101F600066610BE0002001F036FAFFF76BFF0221FB
:101F70009DF80000FEF7B6FD00E0A56160683D54E5
:101F8000F8BDE06880B1401EE661E0602A48A168C3
:101F9000405C491CA1600321FEF7A4FDA068B0F5D8
:101FA000806FEDD1A560F8BDE561F8BD20F000407F
:101FB000C0F1FF40C00F70470FB400B5C1B043AAD5
:101FC0006846429903F068FB6846FEF7C3FD41B0DE
:101FD0005DF814FB726573657420686973746F72C1
:101FE00079000000256C7520256C6C752025662015
:101FF0002566202566202566000000002578000063
:10200000D80700203E3E000070000020D8020020CB
:10201000E86A0000940000200D0A00000D0A556EC9
:102020006B6E6F776E20636F6D6D616E6421202023
:102030002000000000500040D803002010B5D04C14
:102040000521204602F09AF8FC21204602F0A1F872
:1020500001224FF49871002002F008FA4F214E201F
:1020600002F038FABDE81040152000F058B910B55C
:10207000C44C0020608002F05DFA60806088000738
:1020800008D5002002F017FA2178BF4A0A44491CFB
:102090002170107010BD70B5BA4A0C460021517005
:1020A0004006050E152000F047F9210A002002F035
:1020B00009FA284602F014FAE0B2BDE8704000F0D8
:1020C0004CB910B51468FFF7E6FF200E00F045F993
:1020D000C4F3074000F041F9C4F3072000F03DF9D4
:1020E000E0B200F03AF9BDE8104000F03EB907B5A3
:1020F00002AAFFF7E6FF0EBD07B502AAFFF7E1FF50
:102100000EBD10B51446FFF7C6FF02E0641C00F0D8
:1021100024F920780028F9D100F01FF9BDE810401B
:1021200000F023B92DE9F041964E0D4600211446EA
:1021300031704006070E152000F0FEF8290A002035
:1021400002F0C0F9E9B2002002F0BCF9384602F012
:10215000C7F98E4881888907FCD10022214638467C
:1021600002F0D1F9152000F0DAF83078A042FCDB5B
:10217000BDE8F08170B51D461446102A00DD10241C
:102180002246FFF7CFFF00207F4902E00A5C2A5475
:10219000401CA042FADB00202919487070BD10B520
:1021A0000422FFF7BFFF7849C87860F307048878F6
:1021B0004A7860F30F242046097862F3174061F3F0
:1021C0001F6010BD10B50422FFF7ACFF6E49C87840
:1021D00060F3070488784A7860F30F242046097872
:1021E00062F3174061F31F6010BD70B5654C0E4679
:1021F000002121704006050E152000F09DF83146A3
:10220000002002F05FF9284602F06AF95F488188F1
:102210008907FCD100220221284602F074F915201A
:1022200000F07DF820780228FCD3574841780078E8
:1022300041EA002070BD70B5524C0E46002121705D
:102240004006050E152000F077F83146002002F018
:1022500039F9284602F044F94C4881888907FCD1B5
:1022600000220221284602F04EF9152000F057F80E
:1022700020780228FCD344484178007841EA0020C5
:1022800000B270BD70B53F4C0E4600212170400673
:10229000050E152000F050F83146002002F012F92A
:1022A000284602F01DF9394881888907FCD10022AF
:1022B0000321284602F027F9152000F030F8207895
:1022C0000328FCD33048017842780906807841EA37
:1022D000024141EA002070BD70B51446294A0E46FD
:1022E000002151704006050E152000F025F83146FA
:1022F000002002F0E7F8210A002002F0E3F8284667
:1023000002F0EEF8214881888907FCD1E1B2002073
:1023100002F0D8F8BDE870401520AFF30080002827
:1023200009DB00F01F02012191404009800000F10B
:10233000E020C0F80011704700280DDB00F01F02FC
:10234000012191404009800000F1E020C0F8801197
:10235000BFF34F8FBFF36F8F70470C498A88920786
:10236000FCD10146002002F0ADB810B51520FFF7F2
:10237000D6FF44F62060401E0028FCDC10BD0000A3
:10238000606000409C010020D80A0020003000401E
:10239000FA480168002908D164218160F8490A7E61
:1023A00042F010020A76012141607047F348002193
:1023B000426812B16422C0E90112F14A137E23F08F
:1023C0001003137601607047ED48007E00F0800036
:1023D00070472DE9F041E94D0446443D296902F07A
:1023E00083FC24D8E748844221DD204602F035FCF6
:1023F000E54EE64F32463B4602F0E0FAE44AE54B52
:1024000002F0DFFA02F010FC84B22146482001F00D
:1024100069FD204602F0E7FBDF4AE04B02F0D1FA0B
:1024200032463B4602F0CAFA02F042FCE860BDE8E0
:10243000F0812DE9F041B0F1804F03DD00204FF035
:10244000804101E002F009FC02F032FC10F1FF4F84
:1024500002D30020014601E002F0FFFB02F028FC5D
:10246000C64CCF4D443CE062216B0029DFD002F026
:10247000F4FB012202F086FB06460F46286C02F0B0
:10248000ECFB32463B4602F0FBFB15D2296CE06ABE
:1024900002F06EF902F0E1FB4FF0FF3202F072FB46
:1024A00005460E46E06802F0D8FB2A46334602F0A5
:1024B000E1F902F0FDFB06E0E16AE06802F006F9EE
:1024C000296C02F055F90546216902F017FC07D284
:1024D0002069FFF77EFFBDE8F041092000F07BBFD7
:1024E0002846BDE8F04174E7A1E708B1012802D110
:1024F000A249443908637047A148007D9F49C0F351
:1025000040104439097DC1F340014840704770B51F
:102510009A489A4C01260068443C80B1984D287E28
:1025200040F080002876206B10B12069FFF751FF42
:1025300015F8480F40F004002870A66070BDFFF742
:1025400027FF266470BD8D4910B5443901280DD090
:1025500000280AD1886BC863012048630020086402
:102560008748017E21F08001017610BD486B08B1DB
:102570000F2007E0087DC0070DD0FFF7BDFF012841
:1025800004D00D20BDE8104000F025BF72B6FFF763
:10259000BEFF62B610BDBDE81040B8E710B5002020
:1025A000FFF7D1FF0E2000F016FF012001F04CFED6
:1025B000BFF34F8F10BD70B5704C0125443C01280E
:1025C00014D003281CD000280FD10122002110466E
:1025D00001F040FE04214FF0E0220020C2F88011FB
:1025E000BFF34F8FBFF36F8F606170BD0122114643
:1025F000104601F02FFE022000F046F9656170BD23
:1026000001210022084601F025FE022000F03CF9DD
:102610000320E9E710B540F203110420FEF70BFA9E
:10262000482001F05AFC5F480078C1075348A0F1E8
:10263000440001D0322101E04FF49671816310BD56
:102640004F48017E41F00801017670474C48017EF9
:1026500021F00801017670472DE9F041474E0C4604
:10266000443E054610F1FF4F1ED2716A02F046FB50
:102670001AD34D4F284657F8241002F07FF807EB85
:102680008401896802F022F802F0BAFAB0F5803FBE
:1026900000D300204CB1012C06D181B25FF00800BC
:1026A000FEF7C9F946F82450C1E681B20920F7E7E0
:1026B0003E4A10B5A0F10A01914202D802F093FA05
:1026C00001E000203A4902F0AFFA2C494439C861D0
:1026D00010BD70B5294C443CA06A02F0BEFA054614
:1026E00031480E46616AC06A02F048F802F0B5FA55
:1026F000304A314B02F065F92A46334602F0BAF807
:1027000002F0D6FA2D49884202DD1F481F4901E038
:1027100002F0A3FA02F0CCFA2949884202DC2948E7
:10272000294901E002F099FA02F0C2FA014620615B
:10273000E06802F0E3FA03D22069BDE8704048E6A1
:1027400070BD10B510F1FF4F05D22049884202DC60
:1027500002F083FA09E01448C06A02F07EFA0246E9
:102760000B460020124902F09EF902F0A1FA03493B
:1027700044394862BDE81040ABE70000E4010020A6
:10278000006000406DEA913F5396218E75B1144070
:1027900075D145175DB46F407B650DAD2B26703F3D
:1027A00010000020640200206802002096860100CC
:1027B00000408F40FCA9F1D24D62503FAC8BA54048
:1027C000B4ED913F357D898BB63DF23F0000FA4470
:1027D00010B510F1FF4F05D2B0F1814F02DC02F0CD
:1027E0003CFA01E000202F4902F062FA2E4988628B
:1027F000BDE810406DE72D4890F8440000F001005E
:10280000704700B5FFF7F7FF274951F8200000BDDA
:1028100070B5254C2649A069884207D2401CA061AA
:10282000E169884202D1A068FFF78DFE606B002548
:1028300098B1E06B401EE06300280EDC1B4810F8E6
:10284000481F21F004010170A56000F033F808B9B9
:10285000FFF7ACFD6563A06BE0631348443041684B
:10286000002910D08168491E816000290BDC0121FC
:10287000C0E9001564218160206C002803D0256424
:10288000BDE8704043E670BD002809DB00F01F0280
:10289000012191404009800000F1E020C0F80011C2
:1028A0007047000000000440A001002000600040CC
:1028B000A0860100FE48007E00F00100704770B560
:1028C000FB4CFC4D50B1012807D1FFF761FD207E84
:1028D00040F0010020760120A86470BD207E20F029
:1028E00001002076FFF770FD08B9FFF75FFD0020BB
:1028F000F2E708B1012801D1EE490865704710B52B
:1029000000231A460321102001F0F6FB492001F0B4
:10291000E4FABDE810404B2001F0EDBA2DE9F04794
:10292000E44E81464FF0FF373946706901F096FF5B
:10293000E14903F0A1FC02F090F9884604464546BF
:10294000484602F08AF93A4602F01CF92B46224624
:1029500001F090FF3A4602F015F902F0A9F9054698
:102960002046D64C41460022234602F02AF8DFF8E2
:1029700050830022434602F096F802F055F987B2E0
:10298000284602F06AF90022234602F01AF80022D3
:10299000434602F088F802F047F981B23A464B20EC
:1029A00001F0BFFAC6F81090BDE8F08710B5C14C31
:1029B000012809D0002806D1FFF7B0FF0020FFF75B
:1029C0007EFF0020606410BD0120FFF778FF01202A
:1029D000F8E708B1012801D1B6490864704770B51D
:1029E000B849B94A0144914221D802F036F9B74DAD
:1029F000B74E2A46334601F0E1FFB64AB64B01F026
:102A0000E0FF02F011F984B22146492001F06AFA90
:102A1000204602F0E8F8B14AB14B01F0D2FF2A4655
:102A2000334601F0CBFF02F043F9A249486170BD83
:102A3000AC49AD4A0144914201D89E498861704732
:102A40002DE9F14FDFF86C928CB0D9F850000028D6
:102A50007ED0A648DFF89CA2DFF89CB2816C446B64
:102A6000406C21F0004620F000400590A0488442D0
:102A7000304612DC02F0F1F85A46A04B01F0A1FFFB
:102A80000022534601F09AFF9D4A9E4B01F099FFA8
:102A900002F00EF980469C4F11E002F0DEF84FF094
:102AA000FF3202F06FF80022534601F087FF974A89
:102AB000974B01F086FF02F0FBF8964F80462046C8
:102AC00002F0CBF80022944B01F075FF0446009011
:102AD0000D46384602F0C1F822462B4601F071FF40
:102AE0000022844B01F0C6FE04460F46304602F039
:102AF000B4F88A4A8A4BCDE9020101F062FFDA4656
:102B00005A46884B01F0B6FE22463B4601F059FF7B
:102B100002F0CEF883464FF03337B6F17C5F1ADC13
:102B200000982C460546404602F097F82A46234670
:102B300001F047FF04460D46DDE9020100227A4B11
:102B400001F039FF3A46794B01F03BFF524600E075
:102B50002BE1774B35E029460098B6F17F5F0546BB
:102B60000C46404619DC02F078F82A46234601F06C
:102B700028FF05460C46DDE9020100225D4B01F00D
:102B80001AFF52465D4B01F01CFF4FF06632694B55
:102B900001F070FE2A46234617E002F05EF82A464E
:102BA000234601F00EFF04460D46DDE90201002236
:102BB000614B01F000FF3A46604B01F002FF00223A
:102BC0005F4B01F057FE22462B4601F0F4FE02F067
:102BD0006FF80446059802F040F85246594B01F050
:102BE000F0FE07460D46204602F037F83A462B46DF
:102BF00001F0E1FE02F05CF807463146584601F06C
:102C0000BDFD02F02AF8504A504B01F033FE02F0AD
:102C10004FF84F4D04462946059801F0AFFD214677
:102C200001F054FD0146384603F012FB8046DDE911
:102C300002015246474B01F0C4FE5246394B01F0A7
:102C400019FE02F035F806462146384601F090FD9F
:102C5000294601F0C5FD059901F08DFD314607902B
:102C600001F034FD01F0F9FFDFF8ECB03B4B5A46C0
:102C700001F0A7FE04460D46384601F0EEFF074678
:102C800022462B46029101F0F5FD02F011F80146B3
:102C9000404603F0DDFA0546304601F0DEFF4FF016
:102CA000FF3201F06FFF06460C46079858E000001F
:102CB000006000400402002000002040E0FFEF40E0
:102CC0000000044092156EC03EA113015396218E60
:102CD00075B1144075D145175DB46F407B650DAD7E
:102CE0002B26703F999919C09999B90010000020BE
:102CF0000000C8410000F03F9A9999999999D93FED
:102D00003BDF4F8D976E723F6F12833AFA7E6ABC3B
:102D10007493683F6F12833B000039407B14AE47C9
:102D2000E17A943F9999C93F0000E03F3333D33FA4
:102D30009999FD3F666600400000F83F3333E33F5A
:102D4000000002409999A93FB81E85EB51B8BE3FDB
:102D500048E17A3F9999B93F465D6BEF5355D53FAE
:102D600001F07BFF3246234601F084FD5A46F94BC1
:102D700001F027FE02460B463846029901F07AFD23
:102D800001F096FF0146284603F062FA01F065FF64
:102D90005246F14B01F06EFD01F08AFF0146D9F871
:102DA000180003F055FAFFF71AFE0C980DB0BDE8B5
:102DB000F04FB3E570B5E94C0546A16801F09EFF00
:102DC00008D82846E16801F08FFF03D8284601F0B3
:102DD00044FF01E00020E24901F06AFF606070BD3D
:102DE00010B510F1FF4F05D2DE49884202DC01F038
:102DF00034FF01E00020DC4901F05AFFD7490862A6
:102E000010BD2DE9F041074602F058FCD34DD34CDC
:102E1000143D48B1A7F50000666AB0F1804F08D8AC
:102E2000384601F01AFF06E00020E8606062BDE865
:102E3000F081CE48CE4901F03BFF0146606230464A
:102E400001F0CEFCE96801F099FCE860EFE710B50D
:102E500010F1FF4F05D2C349884202DC01F0FDFEAC
:102E600001E00020014601F023FFBC49886210BD4B
:102E7000C04910B5884205D8B0F5000F02DA01F05C
:102E8000ECFE02E000204FF0404101F011FFB34999
:102E9000C86210BD10B510F1FF4F05D2B649884287
:102EA00002DC01F0DAFE01E00020B44901F000FF8D
:102EB000AA49086310BDB249B24A10B50144914213
:102EC00002D801F0CAFE01E00020AF4901F0F0FE97
:102ED000A249886010BDAA49AA4A10B5014491428E
:102EE00002D801F0BAFE01E00020A84901F0E0FE9E
:102EF0009A49C86010BDA64910B5884205D8A549B1
:102F0000884202DC01F0A9FE01E00020014601F048
:102F1000CFFE9249C86410BD2DE9F84FDFF878B2B2
:102F20009BF80000012874D19C48006801F04AFE1B
:102F300000229B4B01F045FD01F0BAFE874C06468E
:102F40004FF0010A656D0AFA05F001F032FE3146D4
:102F500001F014FC4FF48051B0F17D5F02DC914A26
:102F6000904202D985B16D1E08E0B0F17A5F0BDAAC
:102F700010F1834F08D2072D06D26D1C2A010023C1
:102F80008948656500F0E0FF304601F066FEDFF835
:102F90001C82894605460022434601F00FFD074684
:102FA0000E46284649460022434601F063FCDFF8FE
:102FB000B09100224B4601F004FD3A46334601F041
:102FC00072FD01F075FE7A49884202DD00207949E0
:102FD00001E001F042FE01F06BFE6949494288427E
:102FE00002DA0020744901E001F037FE01F060FED2
:102FF0002060216CC9B17149D1E906218A4214D9F6
:10300000E16801F07BFE05D20020FFF79CFA072063
:1030100009E0E2E0A168206801F066FE05D2002028
:10302000FFF791FA082000F0D6F9206801F015FEAC
:10303000054600224B46009101F01CFC06460F4657
:10304000284600224B46009901F0B5FC0022574B60
:1030500001F0B7FC32463B4601F025FD01F028FEA9
:103060008046606801F0F9FD054600224B4600915C
:1030700001F000FC06460F46284600224B46009908
:1030800001F099FC0022494B01F09BFC32463B4683
:1030900001F009FD01F00CFE8146404601F0DDFD26
:1030A000074647488846C06C01F0D7FD00223F4BD9
:1030B00001F081FC05460E46E06C01F0CEFD2A468B
:1030C000334601F07EFC05460E46484601F0C5FD3C
:1030D0002A46334601F0CEFB3A46434601F06BFCEC
:1030E00001F0E6FD1D4D0746143D00266860606C4A
:1030F00070B3286820B13946E86801F0E7FAE86063
:103100003846A96801F034FBA16A01F037FB80461C
:10311000606AE96801F032FB81463946206A01F0B5
:103120002DFB494601F0D2FA414601F0CFFAAF60DB
:103130002861E16A01F0D8FD01D2E06A05E0216B67
:10314000286901F0DBFD3DD2206BFFF779FC2E6092
:103150003DE000005355E53F9999A93F0402002046
:103160000088C3400000C842000024409A99999901
:103170009999D93F000090C000009040000008409D
:10318000000006BC005049040088B340004CCD400C
:103190000050C3C70050C3470000002004000020B7
:1031A0000000443E000040BF000003400000F43F28
:1031B00000504348006A084100407F40A0010020C1
:1031C00010000020C5F800A02869FFF739FC012194
:1031D0006D4800F0DCFE8BF80060BDE8F88F70B53C
:1031E0006A49884202DD0020694901E001F035FDAD
:1031F00001F05EFDB0F17A5F02DA0020654901E07E
:1032000001F02BFD01F054FD634D0446296B01F0E4
:10321000B5FA696B01F05AFA01F0F2FC01040020E2
:1032200000F066FF5D48C46170BD2DE9F04103F018
:1032300063F85A4C06463146D4E90D7001F09EFA07
:1032400005463146E06B01F099FA314601F096FAF5
:10325000314601F093FA04462946384601F036FA21
:10326000214601F033FA01F0F8FC02460B4600203B
:103270004B4901F018FC4FF066324A4B01F0FAFA64
:10328000BDE8F04101F014BD2DE9F05F434F064663
:10329000F86B01F0E2FC8B4604465D46304601F0D7
:1032A000DCFC4FF066323F4B01F085FB02460B46DB
:1032B00000203B4901F0F7FB06468846786B01F099
:1032C000CCFC3246434601F076FB2B46224601F009
:1032D000EAFB01F0EDFC01F0C0FC8A4605460E4613
:1032E0006FF0010201F04EFC33462A4601F069FB03
:1032F000804689462046594600222B4B01F061FB4F
:1033000006460C46B86B01F0A8FC3246234601F095
:10331000CAFB01F0CDFC254903F0B6F801F09DFC95
:1033200042464B4601F0A6FA01F0C2FC03F0BCFB9A
:103330000646284651464FF0FF3201F023FC8846EE
:1033400007464446304601F088FC894605463A4621
:10335000234601F08FFA01F0ABFC154E314603F025
:1033600093F804463A4643462846494601F023FB73
:1033700001F09EFC314603F087F8214601F0F8F990
:10338000BDE8F05F02F0ACBE00000340000020404A
:10339000000004400000D03F68020020040200202A
:1033A0000000F03F661271C000000840000040407D
:1033B000ABAAAA3E0E4801680E48002910F8481F23
:1033C00002D041F0080101E021F0080101707047CE
:1033D0000748006870470121814005480268114391
:1033E0000160E7E702490A6882430A60E2E70000F9
:1033F0005C020020006000402DE9F04100215420D3
:10340000FEF7CDFEFF4CA0F17E51A14202D801F0A3
:1034100024FC01E0FC48FD4901F04AFCFC4D04217C
:1034200028605420FEF7BBFEFA4EFB4FB04204D892
:10343000B84202DC01F011FC01E00020014601F07D
:1034400037FCA86008215420FEF7A9FEA0F17E51A8
:10345000A14202D801F001FC01E0EB48EB4901F088
:1034600027FC68600C215420FEF799FEB04204D876
:10347000B84202DC01F0F1FB01E00020014601F05E
:1034800017FCE86010215420FEF789FEE349E44A66
:103490000144914202D801F0E0FB01E0E148E24939
:1034A00001F006FC286114215420FEF778FEDF4964
:1034B000DF4A0144914202D801F0CFFB01E0002035
:1034C000DC4901F0F5FB686118215420FEF767FE26
:1034D000D949884205D8D949884202DC01F0BDFBB0
:1034E00001E00020014601F0E3FBA8611C2154200B
:1034F000FEF755FED249D34F0144B94202D801F03C
:10350000ACFB02E000204FF0804101F0D1FBE8610C
:1035100020215420FEF743FECB4ECC4CB04204D8C1
:10352000A04202DA01F099FB01E00020014601F01F
:10353000BFFB286224215420FEF731FEC449014418
:10354000B94202D801F089FB01E00020C14901F035
:10355000AFFB686228215420FEF721FEB04204D858
:10356000A04202DA01F079FB01E00020014601F0FF
:103570009FFBA8622C215420FEF711FEB349B64AE6
:1035800049420144914202D801F067FB02E04FF04A
:103590006630B24901F08CFBE86230215420FEF71E
:1035A000FEFDAF490144B1F5CE0F02D801F055FB45
:1035B00001E0AC48AC4901F07BFB28633421542086
:1035C000FEF7EDFDA949AA4A0144914202D801F053
:1035D00044FB02E04FF0FF30A64901F069FB68634D
:1035E00038215420FEF7DBFDA34FDFF89082C2198B
:1035F000424502D801F031FB01E00020A04901F072
:1036000057FBA8633C215420FEF7C9FDB04204D803
:10361000A04202DA01F021FB01E00020014601F0A6
:1036200047FBE86340215420FEF7B9FDB04204D8BF
:10363000A04202DA01F011FB01E00020014601F096
:1036400037FB286444215420FEF7A9FDC2194245E6
:1036500002D801F002FB01E00020894901F028FBBB
:10366000686448215420FEF79AFDB04204D8A04275
:1036700002DA01F0F2FA01E00020014601F018FB45
:10368000A8644C215420FEF78AFDC219424502D895
:1036900001F0E3FA01E00020794901F009FBE86458
:1036A00050215420FEF77BFDB04204D8A04202DA3C
:1036B00001F0D3FA01E00020014601F0F9FA5421AB
:1036C00028650846FEF76BFD6E4AC119914202D883
:1036D00001F0C3FA01E000206B4901F0E9FA6865E6
:1036E00058215420FEF75BFDC219424502D801F073
:1036F000B4FA02E000204FF0804101F0D9FAA86549
:103700005C215420FEF74BFDB04204D8A04202DAFF
:1037100001F0A3FA01E00020014601F0C9FAE865D2
:10372000BDE8F08110B53A4C002154202268FEF724
:10373000DEFC04215420A268FEF7D9FC08215420A5
:103740006268FEF7D4FC0C215420E268FEF7CFFC3F
:10375000102154202269FEF7CAFC1421542062690A
:10376000FEF7C5FC18215420A269FEF7C0FC1C21FD
:103770005420E269FEF7BBFC20215420226AFEF7A8
:10378000B6FC24215420626AFEF7B1FC28215420A3
:10379000A26AFEF7ACFC2C215420E26AFEF7A7FCDB
:1037A00030215420226BFEF7A2FC34215420626B9E
:1037B000FEF79DFC38215420A26BFEF798FC3C21BB
:1037C0005420E26BFEF793FC40215420226CFEF75C
:1037D0008EFC44215420626CFEF789FC4821542061
:1037E000A26CFEF784FC4C215420E26CFEF77FFCB7
:1037F00050215420226DFEF77AFC54210846626D58
:1038000044E0000000409C06C443183F8D07484038
:103810006802002000401CC600401C46E8482EC735
:10382000E848AE067B14AE47E17A843F000060BEF4
:103830000050A30600409F4000409CC600409C46AC
:10384000F5285CC3F528A406CDCCCCBDCDCCCC3DB1
:10385000F5285CC40000E03F3333D3036666EA3FDB
:103860000000D13B6EDBB66DDB4A8CC0000006BBAE
:1038700000C06000FFF8A440F528DCC3F528FC0474
:103880000000F03FF528560800005E40FEF72FFCD0
:1038900058215420A26DFEF72AFCE26D5C21BDE8A0
:1038A00010405420FEF723BC70B541F2584154201B
:1038B000FEF788FCFEF7FCFE4FF4A3515420FEF700
:1038C0006EFCFEF73EFF41F268415420FEF767FCB4
:1038D000FEF77EFF4FF4A0515420FEF773FCF74C27
:1038E000012800D00020F649886041F204415420AC
:1038F000FEF755FC0021FEF7AFFE41F208415420CF
:10390000FEF74DFC0121FEF7A7FE41F20C415420C9
:10391000FEF745FCFEF75DFD41F21C415420FEF729
:103920003EFCFFF75DFA4FF4A1515420FEF737FC3F
:10393000FFF767FA41F224415420FEF730FCFFF70D
:1039400086FA41F230415420FEF729FCFFF790FA45
:1039500041F234415420FEF722FCFFF79BFA41F27A
:1039600028415420FEF71BFCFFF7A5FA41F22C4139
:103970005420FEF714FCFFF7AEFA41F21841542030
:10398000FEF70DFC0546A16801F0B8F908D82846F5
:10399000E16801F0A9F903D8284601F05EF901E0D9
:1039A0000020C84901F084F9606041F23841542098
:1039B000FEF7F5FB606341F23C415420FEF7EFFB5C
:1039C000A0634FF4A2515420FEF7E9FBE06341F2FB
:1039D00044415420FEF7F6FBFEF7FBFF41F248415D
:1039E0005420FEF7EFFBFEF7E1FF41F24C4154207B
:1039F000FEF7D5FBFEF7F3FF41F250415420FEF7EE
:103A0000CEFBFFF7ECFB41F254415420FEF7C7FB1D
:103A1000FFF771FA41F264415420FEF7C0FBFFF753
:103A200007F841F248015420FEF7CCFBBDE8704096
:103A3000FDF720B870B5A24D4FF4A0515420AA68EC
:103A4000FEF75AFB41F2044154202A68FEF74FFB6F
:103A500041F2084154206A68FEF749FB41F20C41EB
:103A60005420EA68FEF743FB944C41F2184154207D
:103A70006268FEF73CFB41F21C415420226AFEF7CB
:103A800036FB4FF4A1515420626AFEF730FB41F23D
:103A900024415420A26AFEF72AFB41F2304154200F
:103AA000E26AFEF724FB41F234415420226BFEF718
:103AB0001EFB41F228415420A268FEF718FB41F298
:103AC0002C415420E268FEF712FB41F238415420A9
:103AD000626BFEF70CFB41F23C415420A26BFEF7F7
:103AE00006FB4FF4A2515420E26BFEF700FB41F2BB
:103AF00044415420226CFEF7FFFA41F24841542021
:103B0000626CFEF7F9FA41F24C4154206269FEF70B
:103B1000EEFA41F250415420E269FEF7E8FA41F230
:103B200054415420E26CFEF7E2FA41F2584154202D
:103B3000EA69FEF7E1FA41F25C4154202A6AFEF795
:103B4000D6FA4FF4A35154206A6AFEF7D0FA41F234
:103B500068415420AA6AFEF7CAFA41F2644154202F
:103B6000A269FEF7C4FA584841F24801026ABDE86A
:103B700070405420FEF7C0BA10B541F22401542021
:103B8000FEF720FB5149524C88421BD14FF4805123
:103B90005420FEF717FB206020214E4800F025FD41
:103BA0004C4B1F2241F204015420FEF7E3FA41F28C
:103BB00054015420FEF706FB6060411C00D1002038
:103BC000606010BD00202060BDE8104042A1414867
:103BD00000F02BBD10B53E4C4FF4805154202268AC
:103BE000FEF78AFA3B4A41F204015420FEF789FAB3
:103BF000364A41F224015420FEF77EFA6268BDE89D
:103C0000104041F254015420FEF776BA314810B505
:103C10002021203000F0E9FC2E4B1F222033BDE88C
:103C2000104041F228015420FEF7A4BA294A41F27B
:103C3000280120325420FEF764BA70B54FF4C05109
:103C40005420FEF7BFFA284C401C41F604012060C6
:103C50005420FEF7B7FA0646002541F60801542025
:103C6000FEF7B0FA014670194D41C4E9020541F66C
:103C70000C015420FEF793FA206141F61001542004
:103C8000FEF78DFA606141F614015420FEF787FAC1
:103C9000A06141F618015420FEF781FAE06170BD81
:103CA00011484FF4C05102685420FEF725BA0E485F
:103CB00041F60C0102695420FEF719BA04020020F3
:103CC000A00100200088C3407000002063D738099D
:103CD00060020020E80A002043544C333030452D68
:103CE000582D582D5858580010000020124841F601
:103CF000100142695420FEF7FAB90F4841F6140149
:103D000082695420FEF7F3B90B4841F61801C269E5
:103D10005420FEF7ECB910B5074C41F604015420CD
:103D2000A268FEF7E9F9E268BDE8104041F6080133
:103D30005420FEF7E1B900001000002010B54FF448
:103D4000F87202214120FEF7C7FA4FF425520E21E6
:103D50004120FEF7C1FA4FF4C0620F214120FEF767
:103D6000BBFA1021BDE810404FF42A524120FEF763
:103D7000B3BA2DE9F0414A4C206C00F06EFF0546C5
:103D80000E46206900F069FF07460C4604214120D9
:103D9000FEF778FA00F00DFF00F05FFF414A424B5A
:103DA00000F00FFE6FF00B0200F0ECFE3A462346E7
:103DB00000F079FE2A46334600F05CFDBDE8F04194
:103DC00000F076BF2DE9F041354CA06C00F045FFC6
:103DD00005460E46606C00F040FF07460C46052184
:103DE0004120FEF74FFA00F0E4FE00F036FF2F4AC4
:103DF0002F4B00F0E6FD6FF00B0200F0C3FE3A46D9
:103E0000234600F0DEFD2A46334600F033FDBDE8D0
:103E1000F04100F04DBF10B506214120FEF70BFA2E
:103E200000F0C7FEBDE810406FF0060100F016BDBF
:103E300070B52048007D400630D40B214120FEF7AC
:103E4000D4F9044600071DD50420FFF7C4FA1A4828
:103E5000406C10B10020FEF7A9FD1848816821B11F
:103E6000406B10B90020FEF76EFB154D154B00207E
:103E7000D5E908219A1A884104D2FFF74CFF0020A7
:103E8000C5E90800E00602D50520FFF7A4FA2006E0
:103E900004D5BDE870400620FFF79DBA70BD000054
:103EA00068020020F168E388B5F8943E9A999999E0
:103EB0009999293F0060004004020020A0010020E1
:103EC00010000020A08601000A22D321FEF704BAC8
:103ED0004FF4F272D121FEF7FFB940F2E512D12181
:103EE000FEF7FAB989050A0D2121FEF7F5B90A2274
:103EF0000521FEF7F1B910B5044603220221FEF7B1
:103F0000EBF92046BDE8104040F203120421FEF711
:103F1000E3B903221146FEF7DFB900220321FEF7C1
:103F2000DBB970B514460A4605460821FEF7D4F9F8
:103F3000224609212846FEF7CFF92846BDE8704001
:103F400010220521FEF7C8B910B5848C02F0F802E2
:103F500024F0F804224382848268604C22400BB132
:103F600042F4802201F4405111438160012010BDD0
:103F700010B54FF4706401F07F0104EA022211438E
:103F80004DF28002134019430184008C10BD8268F9
:103F900011B142F4002201E022F4002283681343AD
:103FA0008360828C01F0070122F0070211438184B3
:103FB000012070470078704700797047806C704727
:103FC000C068704710B58368454C02F470322340D6
:103FD0001A438260828B01F00F0102F47F52114379
:103FE0008183012010BD82683E4B01F440611A407C
:103FF000114381600120704710B583683A4C02F488
:10400000787223401A4301F01F011143816001209F
:1040100010BD02B101710079704710B5848B01F4B5
:10402000E06104F01F04214402F44052114403F003
:10403000C0020A438283012010BD4A0706D50279D7
:1040400042F004020271042280F84420090706D5D8
:10405000017941F008010171302180F844100120FC
:104060007047114319430180012070471F4A0528FA
:104070002ED2DFE800F0030E1520270021B132F820
:10408000F80F40F0010022E032F8F80F00F01E00B7
:104090001DE00029F8D032F8F80F40F0030016E0D8
:1040A00021B132F8F80F40F0040010E032F8F80FB8
:1040B00000F01B000BE00029F8D032F8F80F40F0B8
:1040C0000C0004E032F8F80F21B140F0100010802D
:1040D0000120704700F00F00F9E70000FFCFFF0F4D
:1040E000FF3F0C00FFF30F0000FCFF000000034047
:1040F000204841604068704730B51E4C9D0501D591
:10410000601502E01144084418442080208830BD26
:10411000B2F1807F02D3D00B03220DE0B2F5801FF5
:1041200002D3100A022207E0B2F5802F02D3100951
:10413000012201E0900800220F4B42F01802188083
:104140000D48083002800B4A108840F6DF73184093
:1041500009B140F020001080108870470548002900
:10416000018802D041F4806101E021F48061018086
:10417000012070470000024000040040018001203F
:1041800070470171027203730120704701710120B1
:104190007047017201207047017301207047FF21B1
:1041A0000173017101760120704730B503884C001E
:1041B0000321A1404FF6FF75691A1940A24011442E
:1041C0000180012030BD10B5047901238B40C3F17B
:1041D000FF0323408A40D1180171012010BD10B5A2
:1041E000047A01238B40C3F1FF0323408A40D11896
:1041F0000172012010BD10B5047B01238B40C3F177
:10420000FF0323408A40D1180173012010BD012211
:104210008A40017B11430173017911430171017ED1
:104220001143017601207047007D70470176007EC2
:1042300070470177007F704700F8201F00787047B3
:1042400000F8241F00787047012181401048018048
:104250000120704770B50E4B20F00304103B1C4446
:1042600083071D0F86070F23360FB34061B101216D
:1042700081400748018042F008002168A840994326
:1042800001432160012070BD206898432060F9E758
:1042900030240040114319430182012070470A4332
:1042A00082810120704700797047017201207047B8
:1042B00000887047B1F5005F07D1018A41F40051D1
:1042C0000182018A21F400510182B2F5805F07D199
:1042D000018A41F480510182018A21F480510182D6
:1042E00001207047B1F5005F018A04D021F400512C
:1042F00001820120704741F40051F9E7B1F5805F78
:10430000018A04D021F4805101820120704741F4D8
:104310008051F9E711431943818201207047008BD6
:104320007047000070B5354CA488072505EA542471
:10433000082C14D2DFE804F00406080A0C0E101250
:1043400001240CE002240AE0042408E0082406E02A
:10435000102404E0202402E0402400E08024284DC2
:104360002D88ED0700D064006501264CB4FBF5F400
:10437000B4FBF1F404854FF40066B6FBF5F5214E6D
:104380007543B5FBF4F4B4FBF1F1A1F5006141F420
:10439000084181840021017103F03C0102F0030215
:1043A00011430173007D70BD0029017B04D041F0F1
:1043B00040010173007D704701F03F01F9E7007D86
:1043C0007047027D920602D50170012070470020DF
:1043D00070470078704702B10174007E7047007E1C
:1043E0007047027922F030020A43027101207047BF
:1043F000017101207047007A7047000000200040E2
:10440000442400400024F40010B5164C238803F027
:10441000200343F0400303430B4313432380012055
:1044200010BD114900B10120C1F8140101207047ED
:104430000C4908390880012070470A48001F00888D
:10444000704708481030008870470748D0F80403C8
:1044500008B10020704703494CF6CC40091D088084
:10446000012070478825004000B0044208433D49C0
:1044700010430880012070473A4A012808D032F8DA
:104480004C0F01290ED020F472401080012070479B
:1044900032F84C0F012902D020F47140F5E740F4C6
:1044A0008070F2E740F40070EFE708432D491043B5
:1044B0000885012070472B49012801D0087A7047F0
:1044C000088E7047274A012802D0117301207047D7
:1044D0009186FBE741EA0020224988840120704749
:1044E0004FF6FE7108401F49FF2807D908770622BA
:1044F00002EAD01040F0F000087602E008760020D2
:10450000087701207047491E41EA022215490A82B4
:10451000C2B2FF2807D90A77062202EAD01040F07B
:10452000F100087604E042F00100087600200877E8
:10453000012070470B49012801D088887047888D79
:1045400070470848808A70470649088701207047ED
:1045500010B5044C24F83C0FA1802281A3810120D6
:1045600010BD0000003000401749088810F0180204
:10457000164806D0082A0BD0102A09D0182A0AD1CA
:1045800010E0134A128802F00303124ADA4001E0F5
:104590004FF4004242600988426801F00701CA40B6
:1045A000026070478268F5E70B49002008800649E1
:1045B0000880074A108088808885D5E7034988608D
:1045C000704702488068704700200040C802002001
:1045D000442400400024F40088250040D2B201E0C9
:1045E00000F8012B491EFBD270470022F6E710B5F8
:1045F00013460A4604461946FFF7F0FF204610BD51
:10460000421C10F8011B0029FBD1801A704710B51D
:10461000002200E0521C835C8C5CA34201D1002B81
:10462000F8D1D8B2E1B2401A10BD034611F8012BFF
:1046300000F8012B002AF9D11846704730B505461D
:104640000020034600E05B1C934205D2EC5CC85C92
:10465000201A01D1002CF6D130BD2DE9F05F934630
:104660000F4680460446002601F03CF8D0F8009042
:10467000824614F8015B2DB100F0C2FB0068405D7A
:10468000C007F6D12B2D02D02D2D1AD0641E00218B
:10469000CAF800105A463946204600F0BEFB0146D3
:1046A00027B13868A04201D1C7F80080DAF80000CD
:1046B000022809D0CAF80090700505D54842BDE827
:1046C000F09F46F48066E2E70846F8E7F0B480EA37
:1046D0000102D40F4200B2EB410F02D2024608465B
:1046E00011464A0042D0C30DDDB2C1F3C752AD1A24
:1046F000202D35DAC1F3160141F4000204B1524213
:10470000C5F1200602FA06F12A411044B3EBD05F4E
:1047100023D0C4B1012DA0EBC35009DCF0BC4FF095
:10472000004202EAC352DBB200F5000000F0DABB3F
:10473000400000F1807000EBC350A0F1807040EAAF
:10474000D170490009E0490841EAC071A0EBC350AB
:1047500000F50000400800EBC350F0BC00F0B9BB0E
:104760006142012202EB4101001BF6E7F0BC7047F9
:1047700081F00041AAE780F00040A7E780EA01024B
:1047800010B502F00043400022D04A001FD0010EB5
:1047900001EB1261C0F35600C2F3560240F4000070
:1047A00042F40002A0FB022000047F39140400D070
:1047B000401C50EA124001D44000491EC2B20C060F
:1047C00004EBD010401C4008802A02D003E00020F7
:1047D00010BD20F00100002900DA0020184310BDB0
:1047E00030B480EA010202F0004530F0004221F0CE
:1047F000004013D090B1C30DD40DC2F31601C0F325
:104800001600E41A41F4000140F400027D349142A4
:1048100001D3641C00E04900002C02DA30BC002007
:1048200070474FF400000023914201D3891A0343DB
:1048300040084FEA4101F7D151B1914202D14FF006
:10484000004105E002D24FF0010101E06FF00101EB
:1048500003EBC450284430BC00F03BBB420005D001
:10486000C0F3C7525242914201DC0020704700EB76
:10487000C15070472DE9FE4F804681EA0300C00F0A
:104880000C46009021F0004123F00045B8EB0200F7
:10489000A94105D24046214690461C460B46024699
:1048A00023F00040104347D0270DC7F30A00C3F39D
:1048B0000A510290401A019040286BDAC3F31300AA
:1048C00040F4801B0098924620B10023D2EB030AEB
:1048D00063EB0B0B01985946C0F14002504600F0C3
:1048E0005EFA06460D4650465946019A00F076FAA1
:1048F00010EB08006141002487EA115284EAE77353
:104900001A4340D0009A62B3019A012A4FEA075233
:1049100015DC001B61EB02014FF0004202EA075276
:10492000CDE90042001C41F5801132462B4600F0D3
:1049300063FB03B0BDE8F08F40462146F9E7001B5A
:1049400061EB0201001C41F5801300185B41201847
:10495000A2F5001747EB030140EAD570B6196D4187
:1049600011E06D084FEA360645EAC0754FEA075276
:10497000001B61EB0201001C41F5801149084FEA60
:1049800030000019514132462B4603B0BDE8F04FCC
:1049900000F023BB0098012240000023D0EB02026C
:1049A00063EBE073009821464FEAE074B8EB000037
:1049B00061EB0401E9E783F000435BE781F000412C
:1049C00058E72DE9FE4F81EA030404F0004421F08A
:1049D000004100944FF0000B23F0004350EA010423
:1049E0005ED052EA03045BD0C3F30A54C1F30A5504
:1049F0002C44A4F2F3340194A0FB0254C1F313013C
:104A000041F48011C3F3130343F4801301FB024408
:104A100000FB034E840A970A44EA815447EA83570D
:104A2000A4FB076802958D0A05FB07854FEA932CC6
:104A300004FB0C542705029D4FEA065847EA163737
:104A4000B5EB08056EEB070C870E920E47EA81174F
:104A500042EA8312A7FB0201B6EB0B0164EB0004F0
:104A60002B0D43EA0C335E1844EB1C50DA465146DA
:104A7000E7FB0201C5F313044FEA0B3343EA145377
:104A80004FEA0432019C43EA0603A4F10C040294A9
:104A9000009CCDE900B400F0AFFA03B0BDE8F08FA0
:104AA00000200146F9E72DE9F04D81EA030404F006
:104AB000004B21F0004514464FF0000A23F000415E
:104AC00050EA050220D054EA01021DD0C5F30A576E
:104AD0000246C5F31303C1F31300C1F30A5640F4B1
:104AE000801543F48013A7EB0608101BD64608F286
:104AF000FD3873EB050002D308F1010801E09218BC
:104B00005B41B8F1000F03DA00200146BDE8F08DEB
:104B100000204FF48011064684460EE0171B73EB0D
:104B2000050705D3121B63EB050306434CEA010C92
:104B300049084FEA300092185B4150EA0107EDD175
:104B400052EA030012D082EA040083EA0501084316
:104B500005D0101BAB4106D20122002306E0002243
:104B60004FF0004302E06FF0010253101AEB060011
:104B70004CEB085110EB0A0041EB0B01BDE8F04D86
:104B800000F02BBA70B521F0004303430CD0C1F301
:104B90000A550024D5EB040564EB0403D617AD1ABF
:104BA000B34102DB0020014670BD201841EB0251E9
:104BB00070BDC10F80EAE0700844CA079623002147
:104BC00000F090B90EB5C10F80EAE0700844CA0742
:104BD000002140F233438DE80E000A460B4600F0F8
:104BE0000BFA03B000BD0EB540F233410291002133
:104BF000CDE900110A460B4600F0FEF903B000BDF6
:104C000020F00040C10DC0F3160040F400007F29E1
:104C100001DA00207047962903DCC1F19601C840F3
:104C20007047963988407047C1F30A5210B5C1F3F6
:104C3000130140F2FF3341F480119A4201DA00205F
:104C400010BD40F233439A42A2F2334203DC524297
:104C500000F0B4F810BD904010BD00F0004230F0FC
:104C600000400AD0C10D01F56071C0F3160042EAA0
:104C70000151C208400711437047002001467047A8
:104C800030B5041E71F1000404DB4FF000444042D3
:104C900064EB0101141E73F1000405DB1C464FF0A8
:104CA0000043524263EB0403994208BF904230BD77
:104CB00001F0004330B421F0004150EA010206D077
:104CC0000A0DA2F56072C1F31301002A02DC30BCA8
:104CD00000207047440F44EAC104C100E01830BC12
:104CE00000EBC25000F0F5B8002801DBC0F1004035
:104CF000002901DBC1F1004181427047002801DB3E
:104D0000C0F10040002901DBC1F100418842704739
:104D100030B50B46014600202022012409E021FA8B
:104D200002F59D4205D303FA02F5491B04FA02F588
:104D30002844151EA2F10102F1DC30BD2DE9F05F1F
:104D40000546002092469B468846064681464024FA
:104D50001BE0284641464746224600F02FF85346BE
:104D60005A46C01A914110D311461846224600F007
:104D700016F82D1A67EB01084F4622460120002144
:104D800000F00DF817EB00094E41201EA4F10104BC
:104D9000DFDC484631462A464346BDE8F09F202ADC
:104DA00004DB203A00FA02F1002070479140C2F182
:104DB000200320FA03F3194390407047202A04DBB4
:104DC000203A21FA02F00021704721FA02F3D04084
:104DD000C2F120029140084319467047202A06DBA1
:104DE000CB17203A41FA02F043EAE07306E041FAB9
:104DF00002F3D040C2F120029140084319467047A7
:104E000000487047246E000010B50446FFF7F8FF15
:104E10000068005D00F0010010BD2DE9F05F8246E2
:104E20000078002715468B460AF10104B946302860
:104E300001D09DB113E014F8010B0127782803D0AD
:104E4000582801D045B10AE00DB1102D07D1002737
:104E5000102514F8010B02E0082500E00A250026C1
:104E6000B0460EE005FB080005FB06F1012701EB4B
:104E700010461FFA80F8B6F5803F00D3B94614F803
:104E8000010B294600F08CF90028EBDABBF1000F8A
:104E900005D00FB1641E00E05446CBF80040B9F1D4
:104EA000000F06D000F01EFC02210160C81EBDE804
:104EB000F09F48EA0640FAE77CB50023CDE90033CD
:104EC0000546684600F095F96946284600F026FC3C
:104ED0007CBD0029A8BF7047401C490008BF20F0D6
:104EE0000100704710B4B0FA80FC00FA0CF050EAF0
:104EF000010404BF10BC704749B1CCF1200421FA71
:104F000004F411FA0CF118BF012121430843A3EB6B
:104F10000C01CB1D4FEA00614FEA102042BF002078
:104F200010BC704700EBC35010440029A4BF10BC54
:104F30007047401C490008BF20F0010010BC7047BA
:104F4000F0B4002802DCF0BC00207047C0F3C75169
:104F5000C0F3160040F40000CA0701D14000491E0A
:104F60003F2202EB6105002211464FF4000626FAAB
:104F700001F31344D418844201D8001B1A464000A0
:104F8000491C1729F3DD5100814202D24FF0FF3155
:104F900000E0002102EBC550F0BCFFF79ABF10B54E
:104FA00041000CD0C0F3C751962908DC7E2909DCEA
:104FB00006DB410204D000F0004040F07E5010BDFE
:104FC000002010BDC1F19604C4F1200100FA01F1E6
:104FD000E040FFF77EFFA04010BD10B5141E73F136
:104FE000000408DA401C41F1000192185B411A43A9
:104FF00001D120F0010010BD2DE9F04D92469B46F5
:1050000011B1B1FA81F202E0B0FA80F2203290469A
:10501000FFF7C5FE04460F4640EA0A0041EA0B01CD
:1050200053465A46084313D0114653EA010019D09B
:10503000C8F140025046FFF7C1FE05460E465046F5
:1050400059464246FFF7ABFE084305D0012004E075
:1050500020463946BDE8F08D0020054346EAE0765B
:105060002C4337430A986305E40AA0EB08000022AA
:10507000FD0A44EA47540A3002D500200146E9E718
:10508000010510196941DDE9084500196941BDE8CC
:10509000F04DA2E700F0004220F00040C10DC0F347
:1050A000160040F400007F2901DA0020704796299D
:1050B00003DCC1F19601C84001E096398840002A1E
:1050C000F4D040427047C1F30A52C1F3130140F2D9
:1050D000FF3341F480119A4202DA00200146704702
:1050E00040F233439A42A2F2334202DC5242FFF7CB
:1050F00065BEFFF754BE10B500F0004420F000403C
:10510000C20DC0F3160040F400007F2A07DA7D2AA2
:1051100000DA7D22763A00FA02F1002008E0962AB1
:1051200009DCA2F1760100FA01F1C2F19602D04049
:10513000FFF7CFFE01E0963A9040002C00D04042AD
:1051400010BD002801DBC0F10040002901DBC1F1E6
:105150000041814202D24FF0004004E04FF0005085
:1051600001D14FF0C0404FEA2062EFF3008162F3BB
:105170001F6181F30088704700207047064C074D7F
:1051800006E0E06840F0010394E807009847103417
:10519000AC42F6D3FAF7BCFF10710000207100009A
:1051A0003A2800D2303820F02002412A01D3A2F15F
:1051B0003700884201D34FF0FF3070470FB400230F
:1051C00000B589B00CA900910B996FF00042CB603B
:1051D0001E4B06931E4B07930423CDE901321D4A53
:1051E000089202466B46002000F0CAF809B05DF84C
:1051F00014FB70B586B006464FF0FF300091CDE944
:105200000101002015460C4604903246694604A868
:10521000FFF7D4FF02460498211825B108B10846CB
:1052200000E020462860049800280DD0002A02DD06
:105230000098884208D0081B0094CDE9010432464A
:10524000694604A8FFF7BAFF06B070BDB955000063
:10525000D7550000094E00002DE9FF4F087883B0B4
:105260009946FF2805D0491C2D2804D00024002091
:1052700008E000200BE00124F9E700EB800003EBDD
:105280004000491C0B78FF2BF7D104B140420023AA
:105290000293147819461D462D2C01D02B2C04D1D5
:1052A000521C2D2C13D000240294AA461478FF2CF3
:1052B0000FD00A25A3FB057801FB05814FF0000CF8
:1052C00003FB0C11521CE3194AEB0101EEE7012428
:1052D000EAE7814453EA010002D019F5C87F06DAF3
:1052E00003980021C0E9001107B0BDE8F08F002548
:1052F000AE4E2F46DFF8B882184600F095F9CDE99A
:105300000001B9F1000002DAC9F1000400E004462E
:105310000023A74A1AEB030B42EB045A12E0E00702
:1053200007D02A46334638464146FFF74AFB074630
:1053300088462A46334610461946FFF742FB054683
:105340000E466410002CEAD1DDE90001B9F1000F2E
:105350005A46534606DAFFF7A6FB3A464346FFF79E
:10536000A2FB05E0FFF72DFB3A464346FFF729FB7A
:10537000029A0AB181F00041039AC2E90001B3E741
:105380002DE9FF4F1F468DB0D7E901464FF0FF389A
:105390002E2045464FF000090B90B9696D1C0E9800
:1053A0008847396A824688470028F6D1BAF1FF3F1C
:1053B0000AD024F4D064002E11DDBAF12B0F08D0EE
:1053C000BAF12D0F0BD102E0404611B08DE744F445
:1053D0008064B9696D1C0E9888478246761E6946BE
:1053E000600501D52D2000E02B208DF8000001F193
:1053F000010B0DF1200809E0B9696D1C0E98884772
:1054000082460F9844F40074761E0560002E02DD7B
:10541000BAF1300FF0D00B998A453ED144F08004A8
:1054200006E00F99681CA9F1010944F400740860B2
:10543000B9696D1C761E0E98884782463028F0D0D8
:105440002BE00B998A4505D1200603D444F0800453
:10545000761E18E0504600F09FFA08B30DF11301D4
:10546000761E44F400748B4508D2AAF130000BF884
:10547000010B200607D5A9F1010003E0200602D4A4
:1054800009F101008146A00502D50F99681C08604A
:10549000B9696D1C0E9888478246002ED1DC53E016
:1054A000002E51DDBAF1650F02D0BAF1450F4BD194
:1054B000A00549D5B9696D1C24F44074761E0E9878
:1054C00088478246002E0CDD2B2804D0BAF12D0F20
:1054D00007D144F48074B9696D1C0E9888478246E0
:1054E000761EE00501D52D2100E02B2108F8011BD7
:1054F000CDF82C8021E00DF12901761E44F40074D2
:1055000088450CD2AAF1300010F0FF0088F80000A6
:1055100002D10B99884509D908F1010806E0E00598
:1055200001D5244801E042F20F708146B9696D1C33
:105530000E98884782460F980560002E04DD50467D
:1055400000F02AFA0028D6D1F9690E988847FF2082
:105550008BF8000088F800000020069007904B466A
:105560006A4608A906A8FFF777FEA00502D46FF0E7
:1055700001002AE714F0240F0AD0E00714D1DDE976
:1055800006123868031D3B600068C0E900120BE09A
:10559000DDE90601FFF78CFB0146E00704D138681E
:1055A000021D3A600068016028460EE700001440C2
:1055B0000000F03FF1D8FFFF426842B1016811F8E6
:1055C000013B23B1521EC0E9001218467047012169
:1055D000C160881E704742685AB1C368016843B908
:1055E00083688B4205D0491E521CC0E9001200207E
:1055F00070474FF0FF30704730B5041E71F1000462
:1056000004DB4FF00044404264EB0101141E73F1CF
:10561000000405DB1C464FF00043524263EB0403D9
:105620008B4208BF824230BD0EB540F23342029237
:105630000022CDE900221346FFF7DEFC03B000BDD7
:1056400070B58C1810F8015B15F0070301D110F844
:10565000013B2A1106D110F8012B03E010F8016B71
:1056600001F8016B5B1EF9D12B0705D40023521EF4
:105670000DD401F8013BFAE710F8013BCB1A921C5C
:1056800003E013F8015B01F8015B521EF9D5A1425A
:10569000D8D3002070BD000037B514460846064B2D
:1056A0006A46214600F080F904466946002000F071
:1056B00012FD20463EBD0000D760000041000802F8
:1056C00018BF04200A0E18BF40F001004FF07F42BF
:1056D00032EA010108BF40F00200012808BF05209E
:1056E0007047000000487047D402002000214FF0AE
:1056F0007E50FFF775B80121FFF7B0B8FEF7E6BF9F
:1057000000210846FFF76CB861214FF0E040FFF739
:10571000A5B86FF05E010807FFF7A0B810B5044602
:10572000D1E9000100F002F8206010BDF8B5044690
:105730000D466A4600F0B4FD00987E3000900028C7
:105740001EDC0022134620462946FFF755FF17D0DE
:10575000002140F60800FFF70FFD064620462946C7
:10576000FFF7A6FA044640F6080006EA0001FFF734
:1057700003FD34F0004004BF022000F045F829E0AA
:105780000098FF2828DB00210846FFF7F5FC00F40D
:1057900040060022134620462946FFF771FA8CBFC7
:1057A00000250125022000F02FF84FF0FF4446B1FC
:1057B000002D0CBF4FF400004FF48000B04218BF22
:1057C000084C04210846FFF7D7FC002D04BF84F0E5
:1057D0000040F8BD2046F8BD20462946BDE8F84007
:1057E000FFF766BAFFFF7F7F02E008C8121F08C1FB
:1057F000002AFAD170477047002001E001C1121F52
:10580000002AFBD170470000014908607047000082
:10581000D40200202DE9FF5F82B00021DDE90430D1
:10582000020DDDF840B0034318D044F61050A2F248
:10583000FF3242431514119801281FD0A5EB0B002D
:10584000401C5FEA000A4FF000064E4FDFF8389127
:10585000B046504615D5CAF1000413E01198012452
:105860004AA3012801D16FEA0B010298119AC0E9FD
:105870000031C0E9024206B0BDE8F09FCBF1000064
:10588000DFE704460021404A491842EB0450CDE9C5
:10589000001012E0E00707D032463B46404649463A
:1058A000FFF78FF88046894632463B461046194638
:1058B000FFF787F806460F466410002CEAD1DDE9B1
:1058C0000401DDE90023BAF1000F06DAFFF779F8E9
:1058D00042464B46FFF775F805E0FFF7E4F842460D
:1058E0004B46FFF7E0F804460E460022284BFFF730
:1058F000C7F903D84FF0FF30014607E00022254BDF
:1059000020463146FEF7B6FFFFF7DDFB102409E025
:10591000002C0ADB0A220023FFF710FA039B303227
:105920001A55641E50EA0102F2D1641C039AC4F1B4
:1059300011031444119A012A03D0012208430DD106
:105940000AE0084304D000204FF0110B119072E7D9
:10595000A3EB0B056D1E0DE05B4504DD4FF000026F
:1059600005F1010504E003DA4FF00002A5F101059D
:10597000002AECD002981199C0E90231C0E9004533
:1059800079E70000000014400000F03F3000000004
:105990000000F0430000E03F30380A2801D2012027
:1059A00070470020704700002DE9FF4F95B09B46DF
:1059B0008946064600250FE2252877D10024274690
:1059C000F84A0121059400E0044316F8013F203B0A
:1059D00001FA03F01042F7D130782A2811D06FF085
:1059E0002F033078A0F13002092A16D8059A44F026
:1059F000020402EB820203EB42021044761C059083
:105A0000EFE759F8042B0592002A03DA504244F4D8
:105A10000054059044F00204761C30782E2816D1EC
:105A200016F8010F44F004042A280DD06FF02F025D
:105A30003078A0F13003092B09D807EB870302EB7C
:105A40004303C718761CF3E759F8047B761C3078BB
:105A50006C280FD006DC4C2817D068280DD06A2897
:105A600014D104E0742810D07A280FD10DE044F44A
:105A700000140AE044F4801401E044F44014727805
:105A8000824202D104F58014761C761C3078662898
:105A90000BD013DC582877D009DC002875D04528B6
:105AA000F6D04628F4D047281AD19DE118E06328A3
:105AB00035D0642879D0652812D195E1702873D04B
:105AC00008DC6728F1D069286FD06E280DD06F28C8
:105AD00006D1B5E073282CD0752875D0782874D0FD
:105AE0005A46179990476D1C75E1C4F3025002287D
:105AF00009D003280DD0D9F8001004280DD00D606E
:105B000009F1040967E1D9F80010EA17C1E9005268
:105B1000F6E7D9F800100D80F2E70D70F0E719F8FC
:105B2000041B8DF8001000208DF80100EA460120CA
:105B300003E059F804AB4FF0FF3061074FF000016C
:105B400002D40DE008F101018846B9420FDA804520
:105B5000F8DB1AF808100029F4D108E008F1010177
:105B600088468142FADB1AF808100029F6D1059818
:105B70005B46A0EB080721463846179A00F094FAD6
:105B8000284400EB080507E04DE029E10DE01AF894
:105B9000010B5A4617999047B8F10108F7D25B46B6
:105BA00021463846179A13E142E00A220092C4F3D4
:105BB00002524FF0000A022A08D059F804CB032AF7
:105BC0004FEAEC710AD00DE029E02AE009F1070163
:105BD00021F00702F2E802C1914609E00FFA8CFCBD
:105BE0004FEAEC71042A03D14FFA8CFC4FEAEC71B6
:105BF000002907DA0A460021DCF1000C61EB020102
:105C00002D2202E0220504D52B228DF8042001224A
:105C100003E0E20701D02022F7E7904659E00A218D
:105C200002E010220DE010214FF0000A00910BE07D
:105C300010224FF0000A44F004040827009203E009
:105C400008224FF0000A0092C4F30252022A05D043
:105C500059F804CB0021032A08D009E009F1070113
:105C600021F00702F2E802C1914605E01FFA8CFC20
:105C7000042A01D10CF0FF0C4FF00008220728D5B0
:105C8000702806D0009B83F0100353EA0A0305D066
:105C90000EE040228DF80420012208E05CEA0102B7
:105CA00006D030228DF804208DF80500022290469F
:105CB000009B83F0080353EA0A030AD15CEA01025D
:105CC00001D1620705D530228DF804204FF001087C
:105CD0007F1E582804D034A003900EA802900DE037
:105CE00036A0F9E753466046009AFFF727F8844646
:105CF0000398825C0298401E029002705CEA0100E8
:105D0000F0D1029806A9081A00F1200A600702D50E
:105D100024F4803400E00127574502DDA7EB0A0098
:105D200000E0002000EB0A01009005984144401A71
:105D30000590E00306D45B462146179A059800F0CB
:105D4000B3F90544002706E001A85A46C05D17993B
:105D500090476D1C7F1C4745F6DBE0030CD55B4686
:105D60002146179A059800F09FF9054404E0302079
:105D70005A46179990476D1C0099481E00900029BB
:105D8000F5DC08E0029802995A460078491C029115
:105D9000179990476D1CBAF10001AAF1010AF1DCD4
:105DA00065E10000092801003031323334353637DF
:105DB0003839616263646566000000003031323357
:105DC00034353637383941424344454600000000F7
:105DD00000F058F90544761C307800287FF4ECADCB
:105DE00019B02846BDE8F08F620700D4062709F1F4
:105DF000070222F0070CFCE80223E14603F000480A
:105E00005FEA080C02D00FF2702C0DE05FEA045C30
:105E100002D50FF2682C07E05FEAC47C02D00FF2D3
:105E2000602C01E0AFF2700C4FF0FF3823F000431C
:105E3000CDF850C065280CD006DC452809D046288E
:105E40001DD047283DD13DE0662818D067287ED177
:105E500038E00021112F01DB112000E0781CCDE992
:105E6000000106A90EA8FFF7D5FCDDE90F010E9A87
:105E700003910021009207F1010A04914DE04FF0D7
:105E800000400097CDE9011006A90EA8FFF7C2FC5B
:105E9000DDE90F0203920E9B11990022DDF80CA0A0
:105EA0000093049211B9791C00EB010AB7EB0A00C8
:105EB00004D4C0F1FF3007F1010A0490AAEB0700F7
:105EC000019044E0012F00DA01270021112F01DDAC
:105ED000112000E03846CDE9000106A90EA8FFF721
:105EE00099FCDDE90F010E9A0391002104910092C3
:105EF000BA4621070CD40399514500DA8A46BAF113
:105F0000010F05DD009AAAF10101515C302908D08A
:105F1000B84202DA10F1040F06DA0121CDE90110CE
:105F200015E0AAF10101E9E7002805DC0499014424
:105F30000491AAEB000102E0411C514500DD8A46B4
:105F40000499401A401C01904FF000400290200735
:105F500004D40198504501DBCDF8048000208DF871
:105F60004F0002980DF14F07B0F1004F25D02B20C4
:105F70000E9002984FF0020800280CDA404202907E
:105F80002D200E9007E00A210298FEF7C1FE303165
:105F9000029007F8011DB8F10001A8F10108F2DC38
:105FA00002980028EFD1791E0E980870307800F022
:105FB000200040F0450007F8020D12A8C01B00F1B8
:105FC00007081498007800B1012000EB0A0101983D
:105FD00001EBE07105984144401A401E0590E00332
:105FE00006D45B462146179A059800F05DF80544F3
:105FF0001498007818B15A46179990476D1CE00321
:1060000024D55B462146179A059800F04DF80544C3
:106010001CE00498002807DBDDE90301884203DD6A
:106020000098405C179901E0179930205A46904734
:10603000049805F10105401C04900198401E019050
:1060400004D12E205A46179990476D1CBAF10001D1
:10605000AAF1010ADDDC05E017F8010B5A46179991
:1060600090476D1CB8F10001A8F10108F4DC5B4613
:106070002146179A0598ABE62D0000002B00000082
:10608000200000002DE9F041044600251E46174679
:10609000880404D405E039462020B0476D1C641EF6
:1060A000F9D52846BDE8F0812DE9F04104460025E8
:1060B0001E469046C80301D5302700E020278804FB
:1060C00004D505E041463846B0476D1C641EF9D53D
:1060D0002846BDE8F0810A68531C0B6010707047B9
:1060E0002DE9F04104464FF019404E49002500EBE0
:1060F000440088424AD84C492046FEF73FFBFEF751
:106100004EFF8046FEF7C6FF064648494046FEF76A
:1061100035FB074646494046FEF730FB2146FEF771
:106120002AFB3946FEF724FB04464249FEF726FBCC
:106130004149FEF7CBFA2146FEF720FB6FF04141C3
:10614000FEF7C4FA2146FEF719FB3C49FEF7BEFAFA
:106150002146FEF713FB0146394806F00304784454
:1061600050F82400FEF70AFB3649794451F8241010
:10617000FEF7ACFA3449794451F82410FEF7A6FA38
:10618000B11085BBBDE8F041FEF768BB4FF0FF41A1
:1061900031EA040018D04FF0CE41B1EB440F84BF78
:1061A0004FF07E50BDE8F0812849B1EB440F28BF85
:1061B0000125A0D20220FFF727FB14F0004F0ED0DC
:1061C000BDE8F041FFF7A5BA204614F5000F04BF63
:1061D0000020BDE8F081BDE8F041FFF78CBABDE8D2
:1061E000F041FFF791BAFEF739FB04000BD0B4F190
:1061F000FF4F0FD0FFF762FA042808BFFFF789FAB4
:106200002046BDE8F0810220FFF7FEFABDE8F0412C
:10621000FFF77FBA0220FFF7F7FABDE8F041FFF77A
:1062200073BA00000000501E3BAAB840F4FD0537C9
:106230000070313E12BB2A3D12BB2A3EFFFF7F3F5A
:10624000AE0A0000920A0000760A00000000A08555
:1062500070B50C460546FEF774FF00F07040B0F1D3
:10626000005F07D024F00040C0F1FF40C00F04BF22
:10627000204670BD284670BD70B50C460546FEF739
:1062800060FF00F07040B0F1004F07D024F00040F4
:10629000C0F1FF40C00F04BF204670BD284670BD4E
:1062A00010B5144600222260114A21F000439342A7
:1062B000A8BF10BD53EA000208BF10BDB3F5801F90
:1062C000A8BF226807DA3622FEF75CFC6FF03502C1
:1062D00021F000432260DFF81CC06FF31E510CEB6D
:1062E00023531A4441F0FF5141F00051226010BD88
:1062F0000000F07F02FCFFFF2DE9F0410026A0F531
:106300000001B1F1FE4F7DD200F500226FF07E0159
:1063100001EBE251C2F3025477184FF07E52A0EB2A
:10632000C15602EB045557EA040047D029463046CF
:10633000FEF7CCF9804629463046FEF719FA414669
:10634000FEF74EFA05460146FEF718FA8046454923
:10635000FEF714FA4449FEF7B9F9064641462846C5
:10636000FEF70CFA3146FEF709FA06463846FEF704
:1063700020FC07463D49FEF701FA3D49794451F8B2
:106380002410FEF7A3F93146FEF7A0F906460121D5
:106390002846FEF763FA3146FEF798F90546384677
:1063A0003449FEF7EBF93449794451F82410FEF7EB
:1063B0008DF92946BDE8F041FEF788B94FF07E51CE
:1063C0003046FEF7D5F905462C49FEF7D7F92C499A
:1063D000FEF77CF92946FEF7D1F92A49FEF776F94E
:1063E0002946FEF7CBF96FF08241FEF76FF90446BC
:1063F00029460846FEF7C2F92146FEF7BFF90146D5
:10640000284600E003E0BDE8F041FEF75FB94FF039
:106410007F42B2EB400F03D2BDE8F041FFF76BB90A
:10642000B0F1FF4F08BFBDE8F081B0F1004F06D9D1
:106430000120FFF7E9F9BDE8F041FFF761B930F05D
:10644000004105D06FF016061721FEF707FA5BE74B
:106450000220FFF7D9F9FFF749F980F00040BDE8C5
:10646000F081000066F1CC3EAAAA2A3FF4FD05386F
:10647000C00800000070313F7408000021ED423E6A
:106480000A1180BEC1ABAA3E2DE9F04D0E46002395
:10649000A0F5000C4FF00071354684B002464FF075
:1064A0007E5401EB45014FF07F48BCF1FE4F80F078
:1064B0009F81B1F1804FC0F0DB81FE490144B1F50D
:1064C000005F40F2A78200F58021C90C01F00F07A0
:1064D000C1F307117F39A2EBC15501EB030B38461D
:1064E000FEF767FB6FF00301FEF7B8F94FF07E513E
:1064F000FEF7ECF8014602902846FEF739F90190C4
:1065000028460299FEF7E2F800F5006A6FF30B0ADD
:10651000009051460298FEF72BF92946FEF7D6F86F
:1065200002904FF07E500099FEF75AF90146009014
:106530000198FEF723F900F500656FF30B05284677
:106540000299FEF71BF9029051462846FEF716F90C
:106550000199FEF710F90299FEF70AF90099FEF782
:106560000DF9014601902846FEF7B0F80146029069
:10657000FEF704F98246D049FEF700F9CF49FEF74D
:10658000A5F85146FEF7FAF8824600212846FEF7A4
:1065900065F9009051460298FEF7F0F80546002193
:1065A0000198FEF75BF92946FEF790F8824601460E
:1065B0000098FEF78BF800F500656FF30B05294690
:1065C0000098FEF7D5F85146FEF780F88246BC49A0
:1065D0002846FEF7D3F80090BA495046FEF7CEF8A9
:1065E0008246B9492846FEF7C9F85146FEF76EF8CB
:1065F000824601460098FEF769F800F500656FF3E2
:106600000B0529460098FEF7B3F85146FEF75EF8F1
:106610008246AE48784450F8371000EBC70001912D
:1066200047684FEA0B10FEF7C4FA0090394650460F
:10663000FEF74CF82946FEF749F80199FEF746F8AF
:106640000099FEF743F800F5006B6FF30B0B58460B
:106650000099FEF78DF80199FEF78AF82946FEF7B2
:1066600087F83946FEF784F85146FEF784F806F5B8
:10667000006782466FF30B0739463046FEF778F81D
:10668000002100900846FEF777FD00F00C06394621
:106690005846FEF773F8054620F00040B0F18B4FE6
:1066A0000ADDB8EB400F07D34FF08B4060F31E05B7
:1066B0002F464FF0000A1FE038460099FEF706F813
:1066C0005146FEF75BF8074658460099FEF756F824
:1066D0003946FDF7FBFF824601462846FDF7F6FFE7
:1066E00000F500676FF30B0739462846FEF740F8C0
:1066F0005146FDF7EBFF824631460C20FEF73CFD8C
:1067000051463846FDF7E2FFFEF7F5FC0646051157
:10671000FEF74FFA3946FEF72EF85146FDF7D6FF41
:1067200007466B49FEF72AF86A49FDF7CFFF39465D
:10673000FEF724F86849FDF7C9FF3946FEF71EF851
:106740000146664806F00F06784450F82600FEF72A
:1067500015F86349794451F82610FDF7B7FF6149F0
:10676000794451F82610FDF7B1FF05F17D01FC29B0
:1067700008D22946FEF772F804B02146BDE8F04D74
:10678000FDF7FCBF05F1BF01B1F5BF7F16D8294663
:10679000FEF764F82146FDF7F1FF0546B8EB450F1B
:1067A0001AD068000CD02846FEF788FF042808BFDE
:1067B000FEF7AFFF284604B0BDE8F08D002D0BDAE0
:1067C0000220FFF721F8FEF7A4FF0146204604B09F
:1067D00061F31E00BDE8F08D0220FFF715F8FEF70B
:1067E00093FF0146204604B061F31E00BDE8F08D22
:1067F000B1F1804F3CD300BF00F1FF41B1F1FE4F3A
:1068000021D200BF20F00042C5F3C75110467F29B6
:106810000DDB9729BFF651AEC1F196014FF0010C87
:106820000CFA01F1A1F1010C1CEA050F07D00120BF
:10683000FEF7EAFF04B0BDE8F04DFEF761BF294264
:1068400018BF294C39E641001CBF4FF08071B1EBF5
:10685000400F09D91B21FEF701F802466FF01A0319
:1068600010F0004FCED128E6BCF1FE4F18D224E63E
:10687000B1F1007F0ED336F0004105D006F00041A3
:1068800041F0FC552E46B7E7410018BFB8EB400F6A
:1068900078D8B1E7B1F1807F38BFA5F50006ABD35A
:1068A00020F000416FF0FF4C104C01EB0C03A342B1
:1068B0002FD31DE0001080C07EE24C3EABAAAA3E62
:1068C00000B038423BAA3842D49AB8BB4806000010
:1068D000FC596337C9FF753A1872313D1406000040
:1068E000C80500007C050000000080BFFFFF3F00DE
:1068F00025F000439C44A4450BD3B0F17E5F18BF44
:106900005FEA450C3ED0B1F1FF4F98BFB3F1FF4FA6
:1069100005D904B03146BDE8F04DFEF7EFBEB0F149
:10692000FF4F0FD0C5F3C7517F2909DB972911DA33
:10693000C1F19601012202FA01F14A1E2A4205D054
:10694000002108E015F0004F55D128E0294218BF7A
:10695000012100D1022110F5000F14D020B3B0F1B5
:10696000004F27D010F1814F4ED04FF0FE41B1EBD8
:10697000400F94BF01200020012101EBE571884206
:1069800039D10CE040E015F0004F02D0012936D09B
:1069900031E0012902BF3F4804B0BDE8F08D4FF05F
:1069A000FF4004B0BDE8F08D15F000400ED104B0FA
:1069B000BDE8F08DB5F1FF4F1DD015F5000F05D0E6
:1069C00015F0004F14D009B1012907D00220FEF7BD
:1069D0001BFF04B0BDE8F04DFEF788BE0220FEF7B5
:1069E00013FFFEF783FE04B080F00040BDE8F08D99
:1069F00009B1012903D004B00020BDE8F08D04B036
:106A00004FF00040BDE8F08D04B04FF07E50BDE87F
:106A1000F08D00BF4FF07E51FDF7AAFE05466FF0E6
:106A20000101FDF71BFF1C49FDF7A5FE2946FDF7F7
:106A3000A5FE4FF07C51FDF79EFE0746294608460D
:106A4000FDF79CFE80F000403946FDF797FE824638
:106A500012492846FDF792FE074611495046FDF7B8
:106A60008DFE82460F492846FDF788FE5146FDF708
:106A70002DFE054601463846FDF728FE00F5006B61
:106A80006FF30B0B59463846FDF772FE2946FDF7AA
:106A90001DFEECE5000080FFABAAAA3E00B0B841A5
:106AA0003BAAB841D49A38BB70B50546FEF748FA00
:106AB000044620F00040C0F1FF40C00F08D025F090
:106AC0000040C0F1FF40C00F04BF0120FEF79CFE54
:106AD000204670BD08B50A4600210091014668466F
:106AE000FEF7EAF9009808BD4F0C0000D90F00002E
:106AF000E70F0000011000008D100000FB100000E7
:106B000071120000FD1200001B1300009F13000013
:106B100091140000B1140000C5140000DF1400003F
:106B2000051500001D1500003D150000631500004F
:106B300089150000AF150000CF150000E315000017
:106B4000031600002316000049160000611600001D
:106B5000E116000025170000431700005B17000036
:106B600087170000B1170000D1170000F1170000CF
:106B7000171800003F1800006718000021190000D6
:106B8000491900007119000099190000DF1900006F
:106B9000251A00004D1A0000751A00009D1A000009
:106BA000B71A0000D11A0000EB1A0000051B000004
:106BB0001F1B0000391B0000531B00006D1B000051
:106BC000871B0000A11B0000B11B0000F31B00008D
:106BD000351C0000791C00008F1C0000D31C000035
:106BE000F31C0000F91D00000B1E00000000000057
:106BF0000000803F0030983F0000B53F0040D73F85
:106C000000000000320A7E397F661E395B991F3909
:106C10000000803FF037983FF304B53FFD44D73F75
:106C2000000000000030F13D0070643E0000A33E13
:106C30000090CF3E0090F83E00400F3F00E0203F24
:106C40000000000015B78337CDE37B380EE1C5386F
:106C500060F69138AF5F0F38E1BC3E3823F4473916
:106C600000000000000000000000B33FB2BE7D3A0B
:106C700000002E40DFCF513800007E40BF51FABAED
:106C800000E0A44019DAC3BA00E0C840C2ED8AB9F6
:106C90000040EB40CD1F2CBA001006412AFFFABA83
:106CA00000C01541DFCFD13700D024419A97703A08
:106CB0000050334189478E3600404141E75B9D38A3
:106CC00000B04E41C00A98B900A05B41558F943A7C
:106CD00000306841DA92C0BA0040744162B3C63AEB
:106CE0000000803F00A0853F00908B3F00C0913F97
:106CF0000030983F00F09E3F00F0A53F0050AD3FB0
:106D00000000B53F0000BD3F0060C53F0020CE3F02
:106D10000040D73F00C0E03F00C0EA3F0020F53F01
:106D2000000000007D36AC397D3C3839EBDCF438AE
:106D3000320A7E39124C26399B6AED39A4EE83392A
:106D40007F661E39F6398A392B426539A48211399A
:106D50005B991F39C3EECD39DDE7C637A5A22F39C0
:106D60000000803FC3AA853FC2958B3FD3C3913FAC
:106D7000F037983F32F59E3FD7FEA53F3F58AD3FD5
:106D8000F304B53FA408BD3F2A67C53F8C24CE3F1E
:106D9000FD44D73FDFCCE03FC7C0EA3F7D25F53F4C
:106DA000004040404040404040404141414141401E
:106DB00040404040404040404040404040404040D3
:106DC0004005020202020202020202020202020262
:106DD0000220202020202020202020020202020267
:106DE00002029090909090901010101010101010BF
:106DF00010101010101010101010101002020202CB
:106E0000020288888888888808080808080808080E
:106E1000080808080808080808080808020202020A
:106E200040000000A16D000049444E3F00000000FA
:106E300075736572646174610000000063616C6960
:106E40006200000069746563000000007673746579
:106E5000630000007674656300000000746A756E5C
:106E600063000000706C6F6164000000697068640A
:106E70000000000070626F617264000074626F61F4
:106E800072640000767273656E736500627261747D
:106E9000650000007361766500000000256620250E
:106EA0006620256620256620256620256620256625
:106EB000202566202566202566202566202566205B
:106EC0002566202566202566202566202566202546
:106ED00066202566202566202566202566202566F5
:106EE000202566006566660073747363666700003C
:106EF000636F6E66696700006C6F67006E74636332
:106F0000616C000073657269616C00006D6F64658F
:106F10006C0000006273656C0000000074696C69AD
:106F20006D000000746D6F646761696E00000000A1
:106F3000646761696E000000696761696E00000046
:106F4000706761696E00000061696E0072746D693E
:106F50006E0000007673746D696E000076746D6962
:106F60006E000000746D696E000000007465636F50
:106F70006E000000687776657273696F6E000000BE
:106F800076657273696F6E006C636B6F6E000000E4
:106F9000696C6D6F6E00000076736C6D6F6E000033
:106FA0006C61736F6E0000007673746F6E0000008A
:106FB000766C646175746F007673746175746F00BC
:106FC000766C64726F700000696C617365720000AA
:106FD00076736C6173657200766C61736572000024
:106FE000657272636C720000657272006C636B7321
:106FF0007473000069627573000000007662757337
:107000000000000073746174757300007274616332
:1070100074000000746163740000000072657365A1
:1070200074000000727473657400000074736574FA
:10703000000000007470726F74000000686973745F
:1070400000000000257520257520257520252E348B
:107050006620252E336620252E356620252E3266A5
:1070600020252E336620252E346620252E346620DA
:10707000252E356620252E336620252E33662025C5
:107080002E346620252E326620252E346620252EAD
:10709000346620257820252E316620252E33662063
:1070A000252E336620252E336620252E3366202597
:1070B0002E366620252E366620252E366620252E75
:1070C000336620252E336620252E326620252E326B
:1070D0006620252E3266202575000000696C6D61E2
:1070E00078000000766C6D617800000072746D614C
:1070F0007800000076746D6178000000746D61782E
:10710000000000006C64656C617900000000000004
:107110002071000000000020D8020000405600004E
:1071200001300413B882010349C84113C201233C52
:107130006E23806F231C701AF00C1A04081AE808DA
:107140001AF8041AA0181AC8041AD8041A88041ABB
:10715000EC041A90041AD0041A98042304711ADC5F
:10716000301AE4041AC0101AB0041A14041A6C0479
:107170001A34141A24041A0C041AFC4C1A2C081A77
:1071800014041A440C1A54041A4C041AA8281AB8E5
:10719000042A548019041A40041A38041A30042AA4
:1071A0004C7019301A64081AFC081A5C082AF45446
:1071B00019081A5C3C1A6C041A480C1A7C081A84C8
:1071C000042AFC2019041A640C1A74041AE4042A10
:1071D00094D019141A74041A0C041A28101A3004C2
:1071E0001A8C042A3CE819142AE01C19C801102D35
:1071F000AC8BA5400481C3E803872040CDCC4C3E36
:107200004B2C0104C13264D913A114401C46144014
:107210009C4564606A461A60681A20041BC03F08D7
:107220006D41CDCCCC5C1AC02D800E40197F933AB5
:10723000FC1C763904F6B733695C2908E9682D6AC5
:107240003C40420481250AD7233C6BFA447E7119E5
:107250006C2110093333533FDB5662C4E4C8274521
:107260003A802089082AF050493CD324F4000000D9
:0400000500000109ED
:00000001FF
